:0A0000000C9448040C9400000C94CA
:10000A0000000C9400000C9400000C94E7040C947B
:10001A0000000C94CD040C9400000C9400000C9485
:10002A0000000C9400000C94AD180C9400000C9481
:10003A0000000C9400000C9400000C9400000C9436
:10004A007A040C9400000C9400000C9400000C94A8
:10005A0000000C9400000C9400000C9400000C9416
:10006A0000000C9400000C9400000C9400000C9406
:10007A0000000C9400000C9400000C9400000C94F6
:10008A0000001027E80364000A00010000100001C4
:10009A00100001002020202020CFD0CECFD3D1D2F3
:1000AA00C8D2DC202020202000002020202020CDC3
:1000BA00C0D1D2D0CEC8D2DC2020202020200000FF
:1000CA002020202020CFD0CECFD3D1D2C8D2DC203E
:1000DA002020202000002020202020CDC0D1D2D0F6
:1000EA00CEC8D2DC20202020202000002020202082
:1000FA0020CFD0CECFD3D1D2C8D2DC20202020200E
:10010A0000002020202020CDC0D1D2D0CEC8D2DC01
:10011A0020202020202000002020202020CFD0CE08
:10012A00CFD3D1D2C8D2DC2020202020000020202A
:10013A00202020CDC0D1D2D0CEC8D2DC2020202091
:10014A0020200000202020202020202020202020E5
:10015A00202020202020202000202020CFD0CED6F2
:10016A00C5D1D120D0C0C1CED2DB20202000202092
:10017A002020CDCEC2C0DF20CFC0C9CAC0202020D7
:10018A00200020CFD0CEC4CECBC6C5CDC8C520CF87
:10019A00C0C9CAC8202000202020C4CECF2E20CD1E
:1001AA00C0D1D2D0CEC9CAC820202000C2CDC5D85D
:1001BA00CDC5C520CFCEC4CACBDED7C5CDC8C520D4
:1001CA0000202020202ACFCEC4CACBDED7C5CDCE70
:1001DA002A202020200020202ACDC520CFCEC4CA24
:1001EA00CBDED7C5CDCE2A2020200020202020D04B
:1001FA00C5C6C8CC20D0C0C1CED2DB20202020006A
:10020A00202020202020D1D2C0CDD6C8DF20202017
:10021A002020202000C2C5D0D5CDC8C920CDC0C35A
:10022A00D0C5C2C0D2C5CBDC00202020CFCEC4CEE0
:10023A00C3D0C5C220CFCBC0D2DB202020002020D3
:10024A00202020D0C5C1CECBCBC8CDC320202020B2
:10025A00200020202020D0D3D7CDCEC920D0C5C69B
:10026A00C8CC2020202000202020CFD0CED4C8CB3C
:10027A00DC20CFC0C9CAC82020202000202020208E
:10028A0020536E36332F506233372020202020200F
:10029A00002020202020202020536E41672020208B
:1002AA002020202020002020202020CFD0CED4C8FB
:1002BA00CBDC2030202020202020002020202020DD
:1002CA00CFD0CED4C8CBDC20312020202020200063
:1002DA002020202020CFD0CED4C8CBDC2032202032
:1002EA0020202020002020202020CFD0CED4C8CB10
:1002FA00DC2033202020202020002020202020CF96
:10030A00D0CED4C8CBDC20342020202020200020CE
:10031A0020202020CFD0CED4C8CBDC2035202020EE
:10032A002020200020CFD0CED4C8CBDC20CFCEC412
:10033A00CEC3D0C5C2C0202000202020CFD0CED42A
:10034A00C8CBDC20C2C5D0D5C0202020200020CFB9
:10035A00D0CED4C8CBDC20D0C5C1CECBCBC8CDC380
:10036A00C0200020CDC0D1D2D0CEC9CAC020CFD0A3
:10037A00CED4C8CBDF20200020202054552B253492
:10038A0075B0432020200020202020CCC5D1D2C027
:10039A0020CFC0C9CAC82020202020002020202029
:1003AA00D2C5CCCFC5D0C0D2D3D0C02020202020E7
:1003BA00002020202020204B3D253275202020209F
:1003CA002020202000C2C5D0D5CDC5C3CE20CDC0A7
:1003DA00C3D0C5C2C0D2C5CBDF002020202020CA8E
:1003EA002DCFD0CED4C8CBDF202020202020002043
:1003FA0020204D41583D2533752000202020202003
:10040A00CCCED9CDCED1D2DC20202020202000CDC8
:10041A00C8C6CDC5C3CE20CDC0C3D0C5C2C0D2C503
:10042A00CBDF0020202050572025347520202000C3
:10043A002020202020CCCED9CDCED1D2DC20202025
:10044A002020002020202AC2D0C5CCDF20CFC0C95E
:10045A00CAC82A20202020005425337520D1C5CAB5
:10046A00202020205425327520D7C0D120002020FA
:10047A0020204D41583D2533752020202020202062
:10048A002000202020202020CCCED9CDCED1D2DCF5
:10049A00202020202020002020D2C5CCCFC5D0C0CB
:1004AA00D2D3D0C020C2CACB2E20200020202020A8
:1004BA00202054454D50253375202020002020202F
:1004CA0020202020CFCBC0D2DB20202020202020BB
:1004DA002000D2C5CCCFC5D0C0D2D3D0C020CDC089
:1004EA00C3D0C5C2C000202020D0C5C6C8CC20CAEF
:1004FA00CECDD2D0CECBDF2020200020202020203D
:10050A002AC2CACBDED7C5CD2A202020202020002F
:10051A0020202020202AC2DBCACBDED7C5CD2A2044
:10052A00202020200020D4D3CDCAD6C8DF20C4CEB4
:10053A00CDC0C3D0C5C2C02020002020202020C4A6
:10054A00CECDC0C3D0C5C2C020202020202000208C
:10055A002020D2C5CCCF2EC4CECDC0C3D0C5C2C0F8
:10056A00202020002020202020E2E5F0F1E8FF20D2
:10057A00332E34202020202000202020C4CECFCEAD
:10058A00CBCDC8D2C5CBDCCDDBC5202020002020B6
:10059A00202020CDC0D1D2D0CEC9CAC82020202048
:1005AA00202000202020202ACFD0CECFD3D1D2C8DD
:1005BA00D2DC2A2020202000202AC4C0D2D7C8CAD0
:1005CA0020312028C2C5D0D5292A2020002AC4C01B
:1005DA00D2D7C8CA20322028CDC8C6CDC8C9292A30
:1005EA002000202020CFD0C5C420D3D1D2C0CDCE68
:1005FA00C2CAC820202000202020202020DFD0CA04
:10060A00CED1D2DC20202020202020002020202033
:10061A00205455253375202020202020002020201A
:10062A00202054442533752020202020200020201B
:10063A0020202020205455253375202020202020DA
:10064A002020002020202020D3D1D2C0CDCEC2C865
:10065A00D2DC2020202020002020CDC0D7C0D2DC30
:10066A0020D0C0C1CED2D320CFCE202000C7C0C454
:10067A00C0CDCDDBCC20D3D1D2C0CDCEC2CAC0CC66
:10068A0000205444253375B0432C2020545525337B
:10069A0075B04300205444253375B0430020202010
:1006AA00CDC0D7C0D2DC20D0C0C1CED2D32020202A
:1006BA0020002020C220D0D3D7CDCECC20D0C5C692
:1006CA00C8CCC520202000543D2025750A47005378
:1006DA003D2025750A53004E3D2025750A57004BCB
:1006EA003D2025750A5600503D332E340A52004CDF
:1006FA003D2025750A68004F3D73740A5300473D33
:10070A0073740A5300523DD1F2E0EDF6E8FF0A573E
:10071A0000523DC2C5D0D50A5700523DCFEEE4EE95
:10072A00E3F0E5E20A5700523DD0E5E1EEEBEBE8F3
:10073A00EDE30A5700523DD0F3F7EDEEE90A570010
:10074A00503D536E36332F506233370A5700503DAF
:10075A00536E41670A5700503DCFF0EEF4E8EBFCC8
:10076A0020300A5700503DCFF0EEF4E8EBFC203180
:10077A000A5700503DCFF0EEF4E8EBFC20320A575E
:10078A0000503DCFF0EEF4E8EBFC20330A5700505E
:10079A003DCFF0EEF4E8EBFC20340A5700503DCF91
:1007AA00F0EEF4E8EBFC20350A5700503DCDE5F2B7
:1007BA000A5700D1D2C0CDD6C8DF202000C2C5D08A
:1007CA00D5202020202000CFCEC4CEC3D0C5C22041
:1007DA0000D0C5C1CECBCBC8CDC30020536E3633B3
:1007EA002F5062333700202020202020536E41678B
:1007FA0000CFD0CED4C8CBDC203000CFD0CED4C8E6
:10080A00CBDC203100CFD0CED4C8CBDC203200CF15
:10081A00D0CED4C8CBDC203300CFD0CED4C8CBDCEA
:10082A00203400CFD0CED4C8CBDC20350048C8C78E
:10083A00202020202A4250454DDF2A2020424550C0
:10084A0058202000505725337520202A2534752A30
:10085A00202050572533750074253375B043207412
:10086A00253375B0432074253375B043000080C02A
:10087A0001002D4E414E000002008105780801005A
:10088A0088057A080000F894EE27ECBBF1E0F5BF82
:10089A00E5BFE0936C00F8E1F1BDE1BD8DE0A2E0B7
:1008AA00BB27ED938A95E9F780E090E1A0E0B1E0FB
:1008BA00ED930197E9F7E2E8F8E0859195910097C1
:1008CA0061F0A591B59105901590BF01F0010590D1
:1008DA000D920197E1F7FB01F0CFEFEFEDBFE0E1F9
:1008EA00EEBFC0E0D5E00C94FB1B0E9415241A93BE
:1008FA000A931BB10CB1A12FB0E0ECE1F0E0EA23BE
:10090A00FB233097E1F4E0917E05F0E0E45BFA4FD7
:10091A000083A0917E05AF5FA0937E05A23319F4F0
:10092A00E0E0E0937E05A0918005AF5FA09380058B
:10093A00A23329F4E0E0E0938005689420F80E944D
:10094A002324E03019F405D0E0934905099119915F
:10095A002BC01A93E0918005E030E1F3E0917F0526
:10096A00F0E0E45BFA4F1081A0917F05AF5FA0939E
:10097A007F05A23319F4E0E0E0937F05F894E09153
:10098A008005E150E09380057894E12F199108954C
:10099A000E9415240E9428240E942F240E94362493
:1009AA000E943D240E944424E991EFBFF991E99104
:1009BA00B991A9919991899179916991F99019902F
:1009CA00099018950E9415240E944821989B4FC0AF
:1009DA000E9476240E947B240E9484240E948924F7
:1009EA00E3E6F1E00E948D240E949124999B04C0C1
:1009FA000E9497240E949C24999902C0A895FCCF32
:100A0A000E94A1249A9B04C00E9497240E94A724B2
:100A1A009A9902C0A895FCCF0E94A1240E9497240B
:100A2A00E33028F0A0E0B0E0E0E00E949C2C0E94B5
:100A3A0097240E94AC2429F40E949124E8E7F1E06B
:100A4A0011C0E130A0E0FA0729F40E949124ECE8F1
:100A5A00F1E008C0E230A0E0FA0741F40E949124D4
:100A6A00E1EAF1E0FA93EA930E949421AFCF0E945F
:100A7A00AF240E949724E23010F00C948A05989BC8
:100A8A0042C00E94B7240E9489240E94BA240E946C
:100A9A007624E6EBF1E00E948D24999B04C00E9423
:100AAA0023240E949C24999902C0A895FCCF0E94F5
:100ABA00A1249A9B04C00E9423240E94A7249A99E5
:100ACA0002C0A895FCCF0E94A1240E942324E230F0
:100ADA0028F0A9E2B1E0E0E00E949C2C0E942324C5
:100AEA00E03031F40E949124EBECF1E00E948D2475
:100AFA000E942324E13031F40E949124E0EEF1E0D7
:100B0A000E948D24BCCF0E94AF240E949724E23019
:100B1A0010F00C94E905989B55C00E9476240E9417
:100B2A007B240E9484240E948924E5EFF1E00E943C
:100B3A008D24999B03C0F30131973F01999902C013
:100B4A00A895FCCF0E94A1249A9B03C0F301319679
:100B5A003F019A9902C0A895FCCF0E94A1240E9445
:100B6A00BD2410F466247724062C072831F40E9449
:100B7A009124EAE0F2E00E948D240E94C22431F41A
:100B8A000E949124EFE1F2E00E948D240E94C72482
:100B9A0031F40E949124E3E3F2E00E948D240E9442
:100BAA00CC2431F40E949124E8E4F2E00E948D24DE
:100BBA000E94BD2431F40E949124ECE5F2E00E94E7
:100BCA008D24A9CF0E94AF240E949724E23010F00E
:100BDA000C94FA06062C072811F00C94FA06989B36
:100BEA0002C10E9476240E947B240E9484240E94CF
:100BFA008924E1E7F2E00E948D2499994A9499990F
:100C0A0002C0A895FCCF0E94A1249A9943949A996C
:100C1A0002C0A895FCCF0E94A124E7E0E41508F4DD
:100C2A0044244420C1F40E9491240E94D1240E94A9
:100C3A00D424A2E6B0E00E94FD240E940425A8E381
:100C4A00B0E00E940D25AAE3B0E00E9414250E949C
:100C5A001B250E942625E1E0E415C1F40E94912497
:100C6A000E942D250E943025A4E6B0E00E94FD24B2
:100C7A000E945925A2E4B0E00E940D25A4E4B0E048
:100C8A000E9414250E9462250E942625E2E0E415AE
:100C9A00C1F40E9491240E946D250E947025A6E647
:100CAA00B0E00E94FD240E949925ACE4B0E00E94C5
:100CBA000D25AEE4B0E00E9414250E94A2250E94F0
:100CCA002625E3E0E415D1F40E949124E5ECF2E054
:100CDA000E948D240E94AD25A2E7B0E00E94FD2467
:100CEA000E94D625A6E7B0E00E940D25A8E7B0E04D
:100CFA000E9414250E94DF250E942625E4E0E415BF
:100D0A00D1F40E949124EAEDF2E00E948D240E941F
:100D1A00EA25A4E8B0E00E94FD240E941326A8E870
:100D2A00B0E00E940D25AAE8B0E00E9414250E94B6
:100D3A001C260E942625E5E0E415D1F40E949124A0
:100D4A00EFEEF2E00E948D240E942726A6E9B0E089
:100D5A000E94FD240E945026AAE9B0E00E940D25B7
:100D6A00ACE9B0E00E9414250E9459260E9426256B
:100D7A00E6E0E415D1F40E949124E4E0F3E00E9455
:100D8A008D240E946426A8EAB0E00E94FD240E94F5
:100D9A008D26ACEAB0E00E940D25AEEAB0E00E94D2
:100DAA0014250E9496260E942625E7E0E415D1F430
:100DBA000E949124E9E1F3E00E948D240E94A12679
:100DCA00AAEBB0E00E94FD240E94CA26AEEBB0E076
:100DDA000E940D25A0ECB0E00E9414250E94D326A3
:100DEA000E942625FCCE0E94DE260E949724E2302D
:100DFA0010F00C945A070E94C72411F00C945A0759
:100E0A000E944821989B4DC00E9476240E947B2410
:100E1A000E9484240E948924EEE2F3E00E948D2439
:100E2A0099998A94999902C0A895FCCF0E94A12405
:100E3A009A9983949A9902C0A895FCCF0E94A124FA
:100E4A00E2E0E81508F48824882061F40E949124DD
:100E5A000E94D1240E94E6260E94F926A4ECB0E062
:100E6A000E940027E1E0E81561F40E9491240E94A3
:100E7A002D250E9408270E94F926ABECB0E00E94BB
:100E8A000027E2E0E81561F40E9491240E946D2592
:100E9A000E941B270E94F926A2EDB0E00E940027BB
:100EAA00B1CF0E942E270E9448210E949724E23047
:100EBA0010F00C94B4070E94C22411F00C94B407E9
:100ECA000E944821989B49C00E9476240E947B2454
:100EDA000E9484240E948924E3E4F3E00E948D2482
:100EEA009999DA94999902C0A895FCCF0E94A124F5
:100EFA009A99D3949A9902C0A895FCCF0E94A124EA
:100F0A00E2E0ED1508F4DD24DD2041F40E9491248D
:100F1A000E94D1240E9434270E943F27E1E0ED1568
:100F2A0061F40E9491240E942D25ABEDB0E00E944D
:100F3A004627ADEDB0E00E943F27E2E0ED1561F4EF
:100F4A000E9491240E946D25AFEDB0E00E944627D1
:100F5A00A1EEB0E00E943F27B5CF0E94DE260E9494
:100F6A009724E23010F00C9442080E94CC2411F02D
:100F7A000C9442080E944821989B7DC00E947624C6
:100F8A000E947B240E9484240E948924E8E5F3E0DD
:100F9A000E948D249999CA94999902C0A895FCCF68
:100FAA000E94A1249A99C3949A9902C0A895FCCF49
:100FBA000E94A124E4E0EC1508F4CC24CC2051F4DE
:100FCA000E9491240E94D1240E944D27A9EEB0E0EC
:100FDA000E945827E1E0EC1581F40E9491240E94B6
:100FEA002D25ABEDB0E00E945F27ADEEB0E00E9488
:100FFA00F926AFEEB0E00E945827E2E0EC1581F442
:10100A000E9491240E946D25A3EFB0E00E945F2701
:10101A00A3EFB0E00E94F926A5EFB0E00E9458279E
:10102A00E3E0EC1591F40E949124E5ECF2E00E94D1
:10103A008D24A9EFB0E00E945F27A9EFB0E00E94DB
:10104A00F926ABEFB0E00E945827E4E0EC1591F4E2
:10105A000E949124EAEDF2E00E948D24AFEFB0E005
:10106A000E945F27AFEFB0E00E94F926A1E0B1E04D
:10107A000E94582781CF0E94DE260E949724E230E0
:10108A0010F00C949808062C072811F00C94980874
:10109A00989B47C00E9476240E947B240E94842445
:1010AA000E9489240E9466270E9491240E9469272F
:1010BA00999B04C00E946F270E947427999902C0C5
:1010CA00A895FCCF0E94A1249A9B04C00E946F2776
:1010DA000E9479279A9902C0A895FCCF0E94A12460
:1010EA000E946F27329720F0A6E0B0E00E947E2788
:1010FA000E946F27309741F40E948327EEE9F0E0BF
:10110A000E943E2E0E9488270E946F27319741F441
:10111A000E948327E4EBF0E00E943E2E0E9488277B
:10112A00B7CF0E94AF240E949724E23010F00C94AB
:10113A00EF080E94C72411F00C94EF08989B48C04E
:10114A000E9476240E947B240E9484240E9489247F
:10115A000E9466270E9491240E946927999B04C0D5
:10116A000E948F270E949C24999902C0A895FCCFBF
:10117A000E94A1249A9B04C00E948F270E94A72440
:10118A009A9902C0A895FCCF0E94A1240E948F2799
:10119A00E23028F0A1E0B0E0E0E00E949C2C0E943E
:1011AA008F27E03041F40E948327EAECF0E00E94A6
:1011BA003E2E0E9488270E948F27E13041F40E9428
:1011CA008327E0EEF0E00E943E2E0E948827B6CFE9
:1011DA000E94AF240E949724E23010F00C94460932
:1011EA000E94C22411F00C944609989B48C00E94A0
:1011FA0076240E947B240E9484240E9489240E94CF
:10120A0066270E9491240E946927999B04C00E9424
:10121A0094270E949C24999902C0A895FCCF0E9409
:10122A00A1249A9B04C00E9494270E94A7249A99F9
:10123A0002C0A895FCCF0E94A1240E949427E23004
:10124A0028F0A2E0B0E0E0E00E949C2C0E949427E3
:10125A00E03041F40E948327E6EFF0E00E943E2E40
:10126A000E9488270E949427E13041F40E94832734
:10127A00ECE0F1E00E943E2E0E948827B6CF0E9441
:10128A00AF240E949724E23010F00C949D090E942A
:10129A00CC2411F00C949D09989B48C00E94762496
:1012AA000E947B240E9484240E9489240E9466272B
:1012BA000E9491240E946927999B04C00E94992741
:1012CA000E949C24999902C0A895FCCF0E94A1244F
:1012DA009A9B04C00E9499270E94A7249A9902C047
:1012EA00A895FCCF0E94A1240E949927E23028F0F9
:1012FA00A3E0B0E0E0E00E949C2C0E949927E03035
:10130A0041F40E948327E2E2F1E00E943E2E0E940D
:10131A0088270E949927E13041F40E948327E8E355
:10132A00F1E00E943E2E0E948827B6CF0E94AF2489
:10133A000E949724E23010F00C94210A062C072808
:10134A0011F00C94210A989B6BC00E9491240E9470
:10135A00BA240E949E270E94A3270E94BA270E94AD
:10136A00BF270E9476240E94C227999B04C00E942C
:10137A00C5270E94CA279A9B04C00E94C5270E94BB
:10138A00D3270E94DC2710F00E942824E42D0E9413
:10139A00AC2429F40E94E427A2E3B0E03EC0E13085
:1013AA00A0E0FA0729F40E94E427ACE3B0E035C0D4
:1013BA00E230A0E0FA0729F40E94E427A6E4B0E0AC
:1013CA002CC0E330A0E0FA0729F40E94E427A8E63B
:1013DA00B0E023C0E430A0E0FA0729F40E94E42731
:1013EA00AAE7B0E01AC0E530A0E0FA0729F40E94A3
:1013FA00E427ACE8B0E011C0E630A0E0FA0729F42F
:10140A000E94E427AEE9B0E008C0E730A0E0FA079E
:10141A0031F40E94E427A0EBB0E00E94942C93CF11
:10142A000E94C72411F40E943D240E94C72411F48B
:10143A000E9428240E94AF240E949724E23010F0D0
:10144A000C94780A0E94C22411F00C94780A989B92
:10145A003EC00E9491240E94BA240E949E270E94A4
:10146A00A3270E94BA270E94BF270E9476240E94BF
:10147A00C227999B04C00E94C5270E94CA279A9B2B
:10148A0004C00E94C5270E94D3270E94DC2710F0BF
:10149A000E942824ED2D0E94AC2429F40E94E427FE
:1014AA00A7EDB0E011C0E130A0E0FA0729F40E94EC
:1014BA00E427ABEDB0E008C0E230A0E0FA0731F46F
:1014CA000E94E427AFEDB0E00E94942CC0CF0E94A6
:1014DA00C72411F40E943D240E94C72411F40E94DB
:1014EA0028240E94AF240E949724E230D0F50E945B
:1014FA00BD24B9F5989B33C00E9491240E94BA2456
:10150A000E949E270E94E9270E94EE270E94F32745
:10151A000E94BA270E94BF270E9476240E94C227EF
:10152A00999B06C00E94EE270E9474270E940228F7
:10153A009A9B06C00E94EE270E9479270E940228E1
:10154A000E94EE27ED32A1E0FA0720F0A3E0B1E015
:10155A000E947E27A3E0B1E00E944627CBCF0E94DB
:10156A00AF240E949724E23010F00C94410B062C11
:10157A00072811F00C94410B0E946F27319711F044
:10158A000C94410B989B76C00E9491240E94BA2425
:10159A000E949E270E9408280E94BA270E941128AA
:1015AA000E9476240E941428999B06C00E9417283C
:1015BA000E9474270E9402289A9B06C00E9417283C
:1015CA000E9479270E9402280E941728B49710F0D7
:1015DA000E941C280E9417283F9710F40E941C287A
:1015EA00E42D0E94AC2429F40E941728A6E5B0E055
:1015FA003EC0E130A0E0FA0729F40E941728A8E5C6
:10160A00B0E035C0E230A0E0FA0729F40E941728BA
:10161A00AAE5B0E02CC0E330A0E0FA0729F40E9462
:10162A001728AEE6B0E023C0E430A0E0FA0729F4B8
:10163A000E941728A0E8B0E01AC0E530A0E0FA0737
:10164A0029F40E941728A2E9B0E011C0E630A0E010
:10165A00FA0729F40E941728A4EAB0E008C0E73084
:10166A00A0E0FA0731F40E941728A6EBB0E00E9426
:10167A00942C88CF0E94AF240E949724E23010F065
:10168A000C94D80B062C072811F00C94D80B0E9446
:10169A006F27319711F00C94D80B989B82C00E9447
:1016AA0091240E94BA240E949E27E9EFF3E0FA935C
:1016BA00EA930E9423280E9428280E94BA270E949F
:1016CA0011280E947624E5E0F4E00E948D24999B7B
:1016DA0004C0A7E3B5E00E9437289A9B04C0A7E399
:1016EA00B5E00E943A28A0913705B0913805A43692
:1016FA00E0E0BE0714F00E943D28A0913805AA2315
:10170A0032F4E0E0F0E0E0933705F0933805E42D99
:10171A000E94AC2429F40E942328A5E0B1E03EC02F
:10172A00E130A0E0FA0729F40E942328A7E0B1E0FB
:10173A0035C0E230A0E0FA0729F40E942328A9E084
:10174A00B1E02CC0E330A0E0FA0729F40E94232874
:10175A00ABE0B1E023C0E430A0E0FA0729F40E942C
:10176A002328ADE0B1E01AC0E530A0E0FA0729F479
:10177A000E942328AFE0B1E011C0E630A0E0FA07EA
:10178A0029F40E942328A1E1B1E008C0E730A0E0D3
:10179A00FA0731F40E942328A3E1B1E00E94942CB5
:1017AA007CCF0E94AF240E949724E23010F00C9460
:1017BA00360C0E94C22411F00C94360C0E94942715
:1017CA00E13011F00C94360C989B49C00E94912488
:1017DA000E94BA240E949E270E9408280E94BA27C3
:1017EA000E9411280E9476240E941428999B06C000
:1017FA000E9417280E9474270E9402289A9B06C0FA
:10180A000E9417280E9479270E9402280E941728FE
:10181A00B49710F00E941C280E9417283F9710F4D2
:10182A000E941C28ED2D0E94AC2429F40E9417283E
:10183A00A9EDB0E011C0E130A0E0FA0729F40E9456
:10184A001728ADEDB0E008C0E230A0E0FA0731F4A5
:10185A000E941728A1EEB0E00E94942CB5CF0E94F6
:10186A00AF240E949724E23010F00C94C00C062C8E
:10187A00072811F00C94C00C0E946F27319711F0C1
:10188A000C94C00C989B6BC00E9491240E94BA24AD
:10189A000E949E270E94E9270E9444280E94F3275B
:1018AA000E94BA270E9449280E9476240E94C227D1
:1018BA00999B02C00E944C289A9B02C00E944F2802
:1018CA000E94522810F00E942F24E42D0E94AC247A
:1018DA0029F40E944428A4E3B0E03EC0E130A0E02D
:1018EA00FA0729F40E944428AEE3B0E035C0E2309A
:1018FA00A0E0FA0729F40E944428A8E4B0E02CC02A
:10190A00E330A0E0FA0729F40E944428AAE6B0E0EE
:10191A0023C0E430A0E0FA0729F40E944428ACE787
:10192A00B0E01AC0E530A0E0FA0729F40E94442882
:10193A00AEE8B0E011C0E630A0E0FA0729F40E9450
:10194A004428A0EAB0E008C0E730A0E0FA0731F482
:10195A000E944428A2EBB0E00E94942C93CF0E94EC
:10196A00C22411F40E9436240E94C22411F40E9457
:10197A002F240E94AF240E949724E23010F00C9486
:10198A001D0D0E94C72411F00C941D0D0E948F2773
:10199A00E13011F00C941D0D989B3EC00E949124D9
:1019AA000E94BA240E949E270E94E9270E94442886
:1019BA000E94F3270E94BA270E9449280E9476248F
:1019CA000E94C227999B02C00E944C289A9B02C07F
:1019DA000E944F280E94522810F00E942F24E82DBE
:1019EA000E94AC2429F40E944428A2ECB0E011C061
:1019FA00E130A0E0FA0729F40E944428A9ECB0E0FB
:101A0A0008C0E230A0E0FA0731F40E944428A0EDB1
:101A1A00B0E00E94942CC0CF0E94C22411F40E940C
:101A2A0036240E94C22411F40E942F240E94AF245B
:101A3A000E949724E23010F00C94850D0E94CC2469
:101A4A0011F00C94850D0E949927E13011F00C9445
:101A5A00850D989B53C00E9491240E94BA240E942B
:101A6A009E270E94E9270E9444280E94F3270E9489
:101A7A00BA270E9449280E9476240E94C227999B6D
:101A8A0002C00E944C289A9B02C00E944F280E94C2
:101A9A005A28A732E2E0BE0710F00E942F24EC2D4C
:101AAA000E94AC2429F40E944428A5EEB0E023C089
:101ABA00E130A0E0FA0729F40E944428ABEEB0E036
:101ACA001AC0E230A0E0FA0729F40E944428A1EFE4
:101ADA00B0E011C0E330A0E0FA0729F40E944428DC
:101AEA00A7EFB0E008C0E430A0E0FA0731F40E94A2
:101AFA004428ADEFB0E00E94942CABCF0E94AF24F3
:101B0A000E949724E23010F00C94050E0E94CC2417
:101B1A0011F00C94050E0E949927E13011F00C94F3
:101B2A00050E989B6BC00E9491240E94BA240E94C1
:101B3A009E27EDE2F4E0FA93EA930E945F280E945E
:101B4A0028280E94BA270E9411280E947624EAE3D4
:101B5A00F4E00E948D24999B06C00E945F280E948F
:101B6A0074270E9402289A9B06C00E945F280E943E
:101B7A0079270E9402280E945F28E536A0E0FA072A
:101B8A0024F0A3EEB0E00E946428A4EEB0E00E9424
:101B9A00802CEE2322F4A3EEB0E00E947E27EC2DE7
:101BAA000E94AC2429F40E945F28A9EEB0E023C069
:101BBA00E130A0E0FA0729F40E945F28AFEEB0E016
:101BCA001AC0E230A0E0FA0729F40E945F28A5EFC4
:101BDA00B0E011C0E330A0E0FA0729F40E945F28C0
:101BEA00ABEFB0E008C0E430A0E0FA0731F40E949D
:101BFA005F28A1E0B1E00E94942C93CF0E94AF2409
:101C0A000E949724E23010F00C94BF0E0E94CC245C
:101C1A0011F00C94BF0E0E949927E13011F00C9438
:101C2A00BD0E989BA5C00E9469280E947B240E9431
:101C3A006C280E94BA240E947624EDE4F4E00E9403
:101C4A008D240E949E27E2E6F4E0FA93EA93E0915B
:101C5A001F05F09120050E947028E0911D05F09162
:101C6A001E050E9470280E9475280E9491240E94D5
:101C7A009E270E948721999B1AC00E9402280E94CF
:101C8A007A283197604070400E948C2CEF5FFF4F9A
:101C9A006F4F7F4FAFE1B5E00E947F280E948528F1
:101CAA0030F40E948D28E0931F05F09320059A9B3B
:101CBA0011C00E9402280E947A28EF5FFF4F6F4FDF
:101CCA007F4F0E948C2C319760407040AFE1B5E0A5
:101CDA000E949628A0911F05B0912005A43FE1E03B
:101CEA00BE0760F0A6E1B0E0E4EFF1E060E070E08A
:101CFA000E948C2CE0931F05F09320059B9B13C038
:101D0A000E9402280E947A28E051FE4060407040FA
:101D1A000E949C280E947F280E94852820F40E9405
:101D2A008D280E94A328CF9B22C00E9402280E94CD
:101D3A007A28E05FF14F6F4F7F4F0E949C280E94E4
:101D4A0096280E947A28E038A1E5FA07A1E06A07F6
:101D5A00A0E07A0760F0A6E1B0E0E0E8F1E561E032
:101D6A0070E00E948C2CE8E1F0E00E94A32859CF91
:101D7A000E94AF240E949724E23010F00C944A0F7C
:101D8A00062C072811F00C944A0F0E946F273197EE
:101D9A0011F00C944A0F989B76C00E9491240E94DD
:101DAA00BA240E949E270E94A8280E94BA270E944D
:101DBA0049280E9476240E941428999B06C00E94F2
:101DCA00B1280E9474270E94B6289A9B06C00E94D6
:101DDA00B1280E9479270E94B6280E94B128B49798
:101DEA0010F00E94BC280E94B1283F9710F40E946C
:101DFA00BC28E42D0E94AC2429F40E94B128ACE549
:101E0A00B0E03EC0E130A0E0FA0729F40E94B12810
:101E1A00AEE5B0E035C0E230A0E0FA0729F40E944E
:101E2A00B128A0E6B0E02CC0E330A0E0FA0729F41C
:101E3A000E94B128A0E7B0E023C0E430A0E0FA078E
:101E4A0029F40E94B128A2E8B0E01AC0E530A0E067
:101E5A00FA0729F40E94B128A4E9B0E011C0E630DB
:101E6A00A0E0FA0729F40E94B128A6EAB0E008C067
:101E7A00E730A0E0FA0731F40E94B128A8EBB0E0FD
:101E8A000E94942C88CF0E94AF240E949724E230AB
:101E9A0010F00C94E10F062C072811F00C94E10FB6
:101EAA000E946F27319711F00C94E10F989B82C022
:101EBA000E9491240E94BA240E949E27E8E7F4E037
:101ECA00FA93EA930E94C3280E9428280E94BA27FC
:101EDA000E9449280E947624ECE8F4E00E948D24AE
:101EEA00999B04C0A9E3B5E00E9437289A9B04C0D5
:101EFA00A9E3B5E00E943A28A0913905B0913A05C4
:101F0A00A436E0E0BE0714F00E94C828A0913A0562
:101F1A00AA2332F4E0E0F0E0E0933905F0933A05C1
:101F2A00E42D0E94AC2429F40E94C328A5E1B1E063
:101F3A003EC0E130A0E0FA0729F40E94C328A7E1D5
:101F4A00B1E035C0E230A0E0FA0729F40E94C328C4
:101F5A00A9E1B1E02CC0E330A0E0FA0729F40E941D
:101F6A00C328ABE1B1E023C0E430A0E0FA0729F4CA
:101F7A000E94C328ADE1B1E01AC0E530A0E0FA073B
:101F8A0029F40E94C328AFE1B1E011C0E630A0E015
:101F9A00FA0729F40E94C328A1E2B1E008C0E73099
:101FAA00A0E0FA0731F40E94C328A3E2B1E00E943C
:101FBA00942C7CCF0E94AF240E949724E23010F028
:101FCA000C943F100E94C72411F00C943F100E94F9
:101FDA008F27E13011F00C943F10989B49C00E9462
:101FEA0091240E94BA240E949E270E94A8280E9437
:101FFA00BA270E9449280E9476240E941428999B95
:10200A0006C00E94B1280E9474270E94B6289A9B93
:10201A0006C00E94B1280E9479270E94B6280E9411
:10202A00B128B49710F00E94BC280E94B1283F97AB
:10203A0010F40E94BC28E82D0E94AC2429F40E94C6
:10204A00B128A7ECB0E011C0E130A0E0FA0729F40A
:10205A000E94B128AEECB0E008C0E230A0E0FA0776
:10206A0031F40E94B128A5EDB0E00E94942CB5CFBE
:10207A000E94AF240E949724E23010F00C94B6100C
:10208A000E94CC2411F00C94B6100E949927E130DA
:10209A0011F00C94B6100E945A280E94272E10F0B4
:1020AA000C94B610989B5BC00E9491240E94BA249B
:1020BA000E949E270E94A8280E94BA270E944928A7
:1020CA000E9476240E941428999B06C00E94B12877
:1020DA000E9474270E94B6289A9B06C00E94B128C3
:1020EA000E9479270E94B6280E94B128B49710F05E
:1020FA000E94BC280E94B1283F9710F40E94BC2875
:10210A00EC2D0E94AC2429F40E94B128A7EEB0E07D
:10211A0023C0E130A0E0FA0729F40E94B128ADEE0D
:10212A00B0E01AC0E230A0E0FA0729F40E94B12810
:10213A00A3EFB0E011C0E330A0E0FA0729F40E944F
:10214A00B128A9EFB0E008C0E430A0E0FA0731F402
:10215A000E94B128AFEFB0E00E94942CA3CF0E9456
:10216A00AF240E949724E23010F00C944711062CF9
:10217A00072811F00C9447110E946F27319711F02C
:10218A000C944711989B7CC00E9491240E947B2446
:10219A000E9489240E9411280E947624E1EAF4E030
:1021AA000E948D240E949E270E94CF280E94D82830
:1021BA000E949E270E948721999B06C00E94DF28C1
:1021CA000E9474270E9402289A9B06C00E94DF2858
:1021DA000E9479270E9402280E94DF28EB3FA0E094
:1021EA00FA0720F0AEE2B0E00E947E27E42D0E94BA
:1021FA00AC2429F40E94DF28A0E5B0E03EC0E1301B
:10220A00A0E0FA0729F40E94DF28A2E5B0E035C071
:10221A00E230A0E0FA0729F40E94DF28A4E5B0E042
:10222A002CC0E330A0E0FA0729F40E94DF28ACE6CC
:10223A00B0E023C0E430A0E0FA0729F40E94DF28C6
:10224A00AEE7B0E01AC0E530A0E0FA0729F40E9430
:10225A00DF28A0E9B0E011C0E630A0E0FA0729F4CF
:10226A000E94DF28A2EAB0E008C0E730A0E0FA073F
:10227A0031F40E94DF28A4EBB0E00E94942C82CFB4
:10228A000E94AF240E949724E23010F00C94AD1102
:10229A000E94C72411F00C94AD110E948F27E130DF
:1022AA0011F00C94AD11989B51C00E9491240E9488
:1022BA007B240E948924E7ECF4E00E948D240E948A
:1022CA007624ECEDF4E00E948D240E949E270E9461
:1022DA00CF280E94D8280E949E270E948721999B76
:1022EA0006C00E94DF280E9474270E9402289A9B37
:1022FA0006C00E94DF280E9479270E9402280E94B5
:10230A00DF28EB3FA0E0FA0720F0AEE2B0E00E943F
:10231A007E27E82D0E94AC2429F40E94DF28A5EC30
:10232A00B0E011C0E130A0E0FA0729F40E94DF28EA
:10233A00ACECB0E008C0E230A0E0FA0731F40E9449
:10234A00DF28A3EDB0E00E94942CADCF0E94AF2409
:10235A000E949724E23010F00C944612062C0728AB
:10236A0011F00C9446120E946F27319711F00C94C9
:10237A004612989B84C00E94B7240E9489240E9416
:10238A0049280E947624E0EFF4E00E948D24999B6C
:10239A0004C00E94E4280E947427999902C0A89553
:1023AA00FCCF0E94A1249A9B04C00E94E4280E94A8
:1023BA0079279A9902C0A895FCCF0E94A1240E946D
:1023CA00E428329710F00E94E9280E94E428309706
:1023DA0021F40E9491240E94EC280E94E42831975B
:1023EA0021F40E9491240E94EF28E42D0E94AC243B
:1023FA0029F40E94E428A2E6B0E03EC0E130A0E061
:10240A00FA0729F40E94E428A4E6B0E035C0E230D5
:10241A00A0E0FA0729F40E94E428A6E6B0E02CC05E
:10242A00E330A0E0FA0729F40E94E428A2E7B0E02A
:10243A0023C0E430A0E0FA0729F40E94E428A4E8C3
:10244A00B0E01AC0E530A0E0FA0729F40E94E428B7
:10245A00A6E9B0E011C0E630A0E0FA0729F40E942C
:10246A00E428A8EAB0E008C0E730A0E0FA0731F4AF
:10247A000E94E428AAEBB0E00E94942C7ACF0E9432
:10248A00AF240E949724E23010F00C94B2120E94FA
:10249A00C72411F00C94B2120E948F27E13011F078
:1024AA000C94B212989B57C00E94B7240E948924A8
:1024BA000E9449280E947624E0EFF4E00E948D24CD
:1024CA00999B04C00E94E4280E947427999902C02B
:1024DA00A895FCCF0E94A1249A9B04C00E94E428DC
:1024EA000E9479279A9902C0A895FCCF0E94A1243C
:1024FA000E94E428329710F00E94E9280E94E428FA
:10250A00309721F40E9491240E94EC280E94E4282A
:10251A00319721F40E9491240E94EF28E82D0E940D
:10252A00AC2429F40E94F228A4ECB0E011C0E130F6
:10253A00A0E0FA0729F40E94F228ABECB0E008C048
:10254A00E230A0E0FA0731F40E94F228A2EDB0E0EE
:10255A000E949C2CA7CF0E94AF240E949724E230AD
:10256A0010F00C944F13062C072811F00C944F13FB
:10257A000E946F27319711F00C944F13989B88C0D3
:10258A000E94B7240E9489240E9449280E94762426
:10259A00EFE2F5E00E948D24999B04C00E94F7287F
:1025AA000E947427999902C0A895FCCF0E94A12481
:1025BA009A9B04C00E94F7280E9479279A9902C020
:1025CA00A895FCCF0E94A1240E94F728329720F0F8
:1025DA00A8E0B0E00E947E270E94F728309721F4F5
:1025EA000E9491240E94EC280E94F728319721F436
:1025FA000E9491240E94EF28E42D0E94AC2429F421
:10260A000E94F728A6E3B0E03EC0E130A0E0FA0756
:10261A0029F40E94F728A0E4B0E035C0E230A0E037
:10262A00FA0729F40E94F728AAE4B0E02CC0E330A4
:10263A00A0E0FA0729F40E94F728A4E7B0E023C033
:10264A00E430A0E0FA0729F40E94F728A6E8B0E0EF
:10265A001AC0E530A0E0FA0729F40E94F728A8E991
:10266A00B0E011C0E630A0E0FA0729F40E94F7288A
:10267A00AAEAB0E008C0E730A0E0FA0741F40E94F5
:10268A00F728ACEBB0E00E94942C0E94FC2876CF8D
:10269A000E94AF240E949724E23010F00C94F013A9
:1026AA00062C072811F00C94F0130E946F2731971B
:1026BA0011F00C94F0130E94F728309711F00C9443
:1026CA00EE13989B86C00E9491240E94BA240E940D
:1026DA0048210E946928E4E4F5E00E948D240E94C2
:1026EA007624E1EAF4E00E948D240E949E27E6EB1C
:1026FA00F4E0FA93EA930E9403290E9470280E9448
:10270A00D8280E949E270E948721999B06C00E9472
:10271A0003290E9474270E9402289A9B06C00E94DD
:10272A0003290E9479270E9402280E940329EB3F6D
:10273A00A0E0FA0720F0AAE0B0E00E947E27E42D8C
:10274A000E94AC2429F40E940329A8E3B0E03EC009
:10275A00E130A0E0FA0729F40E940329A2E4B0E0DC
:10276A0035C0E230A0E0FA0729F40E940329ACE45C
:10277A00B0E02CC0E330A0E0FA0729F40E94032954
:10278A00A6E7B0E023C0E430A0E0FA0729F40E94EB
:10279A000329A8E8B0E01AC0E530A0E0FA0729F456
:1027AA000E940329AAE9B0E011C0E630A0E0FA07C6
:1027BA0029F40E940329ACEAB0E008C0E730A0E09F
:1027CA00FA0731F40E940329AEEBB0E00E94942C80
:1027DA0078CF0E94AF240E949724E23010F00C9424
:1027EA009114062C072811F00C9491140E946F275B
:1027FA00319711F00C9491140E94F728309711F038
:10280A000C949114989B7CC00E9448210E949124A8
:10281A000E94BA240E949E270E94E9270E94082942
:10282A000E94F3270E94BA270E9449280E94762410
:10283A00E9E5F5E00E948D24999B06C00E940829CB
:10284A000E9474270E9402289A9B06C00E940829A7
:10285A000E9479270E9402280E940829EB3EA1E0E3
:10286A00FA0720F0ACE0B0E00E947E27E42D0E9437
:10287A00AC2429F40E940829AAE3B0E03EC0E13062
:10288A00A0E0FA0729F40E940829A4E4B0E035C0C0
:10289A00E230A0E0FA0729F40E940829AEE4B0E089
:1028AA002CC0E330A0E0FA0729F40E940829A8E71F
:1028BA00B0E023C0E430A0E0FA0729F40E94082916
:1028CA00AAE8B0E01AC0E530A0E0FA0729F40E94AD
:1028DA000829ACE9B0E011C0E630A0E0FA0729F413
:1028EA000E940829AEEAB0E008C0E730A0E0FA0783
:1028FA0031F40E940829A0ECB0E00E94942C82CF07
:10290A000E94C22411F40E9436240E94C22411F4A7
:10291A000E942F240E94AF240E949724E23011F0D3
:10292A000C94CD16989B5CC00E949124EEE6F5E0CB
:10293A000E948D240E947624E3E8F5E00E948D240B
:10294A000E946928E8E9F5E00E948D2499999A94F1
:10295A00999902C0A895FCCF0E94A1249A999394B0
:10296A009A9902C0A895FCCF0E94A124E5E0E91536
:10297A0008F49924992031F40E940D29EDEAF5E032
:10298A000E948D24E1E0E91531F40E940D29E2EC60
:10299A00F5E00E948D24E2E0E91531F40E940D2948
:1029AA00E7EDF5E00E948D24E3E0E91531F40E9499
:1029BA000D29EDE4F4E00E948D24E4E0E91531F4F8
:1029CA000E940D29ECEEF5E00E948D24E5E0E91560
:1029DA0031F40E940D29E1E0F6E00E948D24A2CF95
:1029EA000E942E27E1E0E91559F5989B29C00E941B
:1029FA009E27E6E1F6E0FA93EA930E9410290E94E4
:102A0A0070280E9415290E949E270E948721999B5F
:102A1A0006C00E9410290E9474270E94B6289A9B19
:102A2A0006C00E9410290E9479270E94B6280E9497
:102A3A001029F39720F0AAE2B0E00E947E27D5CFB2
:102A4A000E94B628E2E0E91559F5989B29C00E9430
:102A5A009E27E7E2F6E0FA93EA930E941A290E9477
:102A6A0070280E9415290E949E270E948721999BFF
:102A7A0006C00E941A290E9474270E94B6289A9BAF
:102A8A0006C00E941A290E9479270E94B6280E942D
:102A9A001A29F39720F0ACE2B0E00E947E27D5CF46
:102AAA00E3E0E91559F5989B29C00E949E27E8E3BF
:102ABA00F6E0FA93EA930E941F290E9470280E9466
:102ACA0015290E949E270E948721999B06C00E9471
:102ADA001F290E9474270E94B6289A9B06C00E944A
:102AEA001F290E9479270E94B6280E941F29FD9754
:102AFA0020F0A4E1B0E00E947E27D5CFE4E0E915FA
:102B0A0011F00C949B16989B11C10E949124EDE43C
:102B1A00F6E00E948D24A2E3B0E0E3ECF0E00E942C
:102B2A00942CA4E3B0E00E942429A6E3B0E00E941A
:102B3A002929ACE3B0E0E6EEF0E00E94942CAEE383
:102B4A00B0E00E942429A0E4B0E00E942929A6E46A
:102B5A00B0E0E6EEF0E00E94942CA8E4B0E00E9417
:102B6A002429A0E5B0E0EEE6F0E00E94942CA2E56C
:102B7A00B0E0E3E7F0E00E94942CA4E5B0E0E9E6D7
:102B8A00F0E00E94942CA6E5B0E00E942E29A8E568
:102B9A00B0E00E942E29AAE5B0E00E942E29ACE5F9
:102BAA00B0E00E942E29AEE5B0E00E942E29A0E6F0
:102BBA00B0E00E942E29A2E6B0E00E947E27A4E699
:102BCA00B0E00E947E27A6E6B0E00E947E27AAE433
:102BDA00B0E00E947E27ACE4B0E0E2EDF0E00E94B3
:102BEA00942CAEE4B0E00E943329A4E5B0E00E9440
:102BFA006428A6E6B0E00E947E27A2ECB0E0E0E9F5
:102C0A00F1E00E94942CA4ECB0E0E0E00E949C2C3D
:102C1A00A5ECB0E0E2E8F0E00E94942CA7ECB0E06A
:102C2A00E8E1F0E00E94942CA5EEB0E00E9424298D
:102C3A00A7EEB0E0E8E1F0E00E94942CA9EEB0E043
:102C4A00E0E5F0E00E94942CA0E2B0E0E0EFF0E0D2
:102C5A000E94942CE0E0F0E00E94A328A6E1B0E0F4
:102C6A00E0E0F0E060E070E00E948C2CA7EDB0E0BC
:102C7A00ECEDF0E00E94942CA9EDB0E0E4E1F0E084
:102C8A000E94942CAAE2B0E00E943329ACE2B0E0A0
:102C9A000E943329A4E1B0E0EAE0F0E00E94942C1B
:102CAA0055240E94E928A0E0B0E0E0E00E949C2CB4
:102CBA00662477240E9438290E943F290E944429C9
:102CCA000E944729A8E0B0E00E942929A2E2B0E0C8
:102CDA000E947E27A4E2B0E00E947E27A6E2B0E02E
:102CEA000E947E27A8E2B0E00E947E27A3E0B1E01E
:102CFA00E4EBF0E00E94942C0E94C8280E943D2830
:102D0A00A5E1B1E00E946428A5E0B1E00E94642830
:102D1A00A7E1B1E00E946428A7E0B1E00E9464281C
:102D2A00A9E2B1E0E1E00E949C2CEDCEE5E0E915D4
:102D3A0059F5989B29C00E949E27E8E3F6E0FA938A
:102D4A00EA930E9452290E9470280E9415290E9423
:102D5A009E270E948721999B06C00E9452290E94A1
:102D6A0074270E94B6289A9B06C00E9452290E9484
:102D7A0079270E94B6280E945229FD9720F0A7E2DF
:102D8A00B1E00E947E27D5CF0E9448210E942E27BB
:102D9A00062C072811F00C945517A895989B80C00B
:102DAA000E9491240E94BA240E9476240E945729E4
:102DBA000E9469280E945A290E949E270E945D2922
:102DCA000E9463290E9475280E940D290E949E274D
:102DDA000E9465290E9447290E94FC28E2E3E093A9
:102DEA001005A895E42D0E94AC2439F40E94D4243D
:102DFA000E9404250E941B254CC0E130A0E0FA077E
:102E0A0039F40E9430250E9459250E94622541C04A
:102E1A00E230A0E0FA0739F40E9470250E94992551
:102E2A000E94A22536C0E330A0E0FA0739F40E94D6
:102E3A00AD250E94D6250E94DF252BC0E430A0E0F4
:102E4A00FA0739F40E94EA250E9413260E941C26DA
:102E5A0020C0E530A0E0FA0739F40E9427260E9434
:102E6A0050260E94592615C0E630A0E0FA0739F428
:102E7A000E9464260E948D260E9496260AC0E73088
:102E8A00A0E0FA0761F40E94A1260E94CA260E94C5
:102E9A00D3260E947C2CE0933705F09338057ECF29
:102EAA000E94C22411F00C949717A895989B3AC0D7
:102EBA00A8950E9491240E94BA240E9476240E9416
:102ECA0057290E9469280E945A290E949E270E9417
:102EDA006C290E94D8280E949E270E9465290E9478
:102EEA0047290E94FC280E942F24ED2D0E94AC2421
:102EFA0019F40E9434270EC0E130A0E0FA0721F04D
:102F0A00E230A0E0FA0761F4ABEDB0E00E94462798
:102F1A00ADEDB0E00E947C2CA0E1B0E00E94942CC0
:102F2A00A895C4CF0E94C72411F00C94DE17A89567
:102F3A00989B3FC0A8950E9491240E94BA240E949F
:102F4A0076240E9457290E9469280E945A290E94C1
:102F5A009E270E945D290E94DF280E9470280E94F5
:102F6A0075280E940D290E949E270E9465290E94A9
:102F7A0047290E94FC280E942824E82D0E94AC249C
:102F8A0019F40E94E6260DC0E130A0E0FA0719F410
:102F9A000E94082706C0E230A0E0FA0741F40E9426
:102FAA001B270E947C2CAEE0B0E00E94942CA895CE
:102FBA00BFCF0E94CC2411F00C945718A895989B67
:102FCA0071C0A8950E9491240E94BA240E94762476
:102FDA000E9457290E9469280E945A290E949E2706
:102FEA00EEE9F6E0FA93EA930E9444280E947028D8
:102FFA000E94D8280E949E270E946529A0E2B0E07C
:10300A000E947E270E9447290E94FC28A895EC2D41
:10301A000E94AC2429F40E944D27A9EEB0E03BC0DF
:10302A00E130A0E0FA0759F4ABEEB0E00E945F2766
:10303A00ADEEB0E00E94F926AFEEB0E02CC0E2306F
:10304A00A0E0FA0759F4A1EFB0E00E945F27A3EFCE
:10305A00B0E00E94F926A5EFB0E01DC0E330A0E081
:10306A00FA0759F4A7EFB0E00E945F27A9EFB0E092
:10307A000E94F926ABEFB0E00EC0E430A0E0FA07F8
:10308A0081F4ADEFB0E00E945F27AFEFB0E00E949D
:10309A00F926A1E0B1E00E947C2CA3EEB0E00E94E8
:1030AA00942C8DCF0E94BD2421F5A895989B21C010
:1030BA00A8950E9491240E94BA240E947624E7EAE5
:1030CA00F6E00E948D240E946928ECEBF6E00E944B
:1030DA008D240E949E270E946C290E94D8280E9453
:1030EA009E270E9465290E9447290E94FC28A895CC
:1030FA00DDCF0E949724E030E1F4A5E2B1E00E941E
:10310A007E270E9471290E947429AA24BB240E9446
:10311A003829E0931305F09314050E944429E0E04E
:10312A00F0E00E943F29E0E0F0E0E0931505F0931B
:10313A0016050E949724E23041F4A8E0B0E00E940C
:10314A0029290E942F240E9428240E9448219DC1D7
:10315A000E9415240E9477290E944428EA1BFB0B2F
:10316A00E0932D05F0932E05062C0728B1F40E9452
:10317A007C292CF00E94832912F40E9436240E9492
:10318A007C295CF4A0913605AA2312F40E94362405
:10319A000E94902914F00E9498290E94C22411F4D6
:1031AA000E9436240E94C724E1F40E947C292CF054
:1031BA000E94832912F40E9436240E947C298CF4EE
:1031CA00A0913605AA2312F40E9436240E9490295F
:1031DA0014F00E9498290E949F29E0932705F093F2
:1031EA0028050E94CC2449F40E945A28129728F0F4
:1031FA000E94A42910F00E94A929A0912505B09146
:10320A0026050E94AE29EA1BFB0BE0932F05F093DB
:10321A0030050E94B3290E94E427EA1BFB0BE093C6
:10322A003105F0933205E1E0E515E1F4062C0728B3
:10323A00C9F40E94B8290E94272E54F40E94B82982
:10324A00159734F40E94BD290E94C2290E94C729F9
:10325A000E94DD293CF40E94E2290E94E72912F427
:10326A000E943D24E1E0E515E9F4062C0728D1F493
:10327A000E94DF280E94F029A8F40E94F4290E94E3
:10328A00DF2832960E94F92968F40E94C2290E9416
:10329A00272E40F40E94FD29E436A0E0FA0710F434
:1032AA000E94022AE1E0E51551F50E94C22439F58F
:1032BA000E94F4290E94E229309711F40E940B2AF5
:1032CA000E94122A54F40E94B829159734F40E94D5
:1032DA00BD290E94C2290E94C7290E94DD293CF407
:1032EA000E94E2290E94E72912F40E943D240E94CA
:1032FA00162AA536E0E0BE0714F00E941B2A0E9497
:10330A00C72411F40E943D240E94162AA436E0E044
:10331A00BE0714F00E941B2AE1E0E515D1F40E94D1
:10332A00CC24B9F40E945A28119738F40E945F28D5
:10333A000E94222A11F40E94A9290E945F280E9451
:10334A00162AAE17BF072CF40E94A42910F40E9473
:10335A00262A0E94292A0E94AE29E0932505F09385
:10336A0026050E942F2AE13BA4E0FA0740F00E94BA
:10337A002F240E9428240E9474290E944429E1E0F3
:10338A00E51581F5E3E0F0E06E167F0658F50E9438
:10339A00DF280E94F92920F00E94FD290E9479273E
:1033AA000E94FD29DF010E94272EE0F40E94DF28F7
:1033BA00DF010E94272EB0F40E94FD29E436A0E026
:1033CA00FA0780F40E94022A0E94FD29EC59FF4F55
:1033DA00A0E3B0E00E94942C0E94E428309711F4F4
:1033EA000E94342AE1E0E51511F00C94461A0E9475
:1033FA00B829119714F00C94461AF50131965F0119
:10340A00E2E0F0E06E167F06E0F500240A140B04F1
:10341A0020F4F501EC59FF4F5F01E6E6F0E0EA150A
:10342A00FB0590F00E94C2290E94272E70F4E5E65F
:10343A00F0E05F01EA15FB0541F40E94022A0E94AE
:10344A003A2AAC9A0E943A2AAC980E941F290E94F2
:10345A00402AEA15FB05A8F40E943D240E9436245E
:10346A000E9428240E942F240E9474290E94442921
:10347A0055240E94452A0E94482A0E94482A0E94EE
:10348A00562A0E942F2A0E947927E991EFBFF991C3
:10349A00E991B991A9919991899179916991F99053
:1034AA001990099018951A930A93B89AC09A0E948B
:1034BA005F2AC0980E94672AE0933B05F0933C0577
:1034CA0089E18A95F1F70E94672AE0933F05F09314
:1034DA004005C09AE0913B05F0913C050E946D2A97
:1034EA00DF01CB01E0913F05F09140050E94752A6A
:1034FA00AAE2B0E027C01A930A93A79AAF9A0E9449
:10350A005F2AAF980E94672AE0933D05F0933E0533
:10351A0089E18A95F1F70E94672AE0934105F093C1
:10352A004205AF9AE0913D05F0913E050E946D2A51
:10353A00DF01CB01E0914105F09142050E94752A15
:10354A00ACE2B0E00E947C2C0E94832ADF01CB010E
:10355A00E0E0F0E068EC72E40E94E22DADECBCEC35
:10356A008CEC9DE30E94462DD801882799270E945A
:10357A00682C0E94942D0E94DA2C8F01F80109917F
:10358A00199108950E9428240E942F240E9436240B
:10359A000E943D240E94442408950E942324E0307E
:1035AA0059F4E1E0E51541F4A0914905A33521F468
:1035BA00E9DFE0E0E09349050E942324E03069F462
:1035CA00552059F4A0914905AA3539F4E1E0E09370
:1035DA004A05A0914A05A130E1F3E1EDF6E0FA933C
:1035EA00EA930E94AE290E9470280E94882AE9ED77
:1035FA00F6E0FA93EA930E942F2A0E9470280E940A
:10360A00882AE1EEF6E00E948D2A0E94882AE9EED5
:10361A00F6E0FA93EA930E94942A0E94882AE1EF3C
:10362A00F6E00E94992AE9EFF6E0FA93EA930E94FB
:10363A009F290E9470280E94882AE1E0E51521F45A
:10364A00E1E0F7E00E94992A552021F4E8E0F7E04A
:10365A000E94992AF301309719F4EFE0F7E01BC0B2
:10366A00E130A0E0FA0719F4EBE1F7E014C0E23028
:10367A00A0E0FA0719F4E4E2F7E00DC0E330A0E0B5
:10368A00FA0719F4E1E3F7E006C0E430A0E0FA072C
:10369A0041F4EFE3F7E0FA93EA9380E00E94E6232D
:1036AA002296062C072811F00C949C1BE42D0E94EC
:1036BA00AC2419F40E94A02A3AC0E130A0E0FA072B
:1036CA0019F40E94A32A33C0E230A0E0FA0719F4E1
:1036DA000E94A62A2CC0E330A0E0FA0729F4EFE6FC
:1036EA00F7E00E94992A23C0E430A0E0FA0729F4FF
:1036FA00EDE7F7E00E94992A1AC0E530A0E0FA0740
:10370A0029F4EBE8F7E00E94992A11C0E630A0E01C
:10371A00FA0729F4E9E9F7E00E94992A08C0E73094
:10372A00A0E0FA0721F4E7EAF7E00E94992A0E944A
:10373A00C224A1F4ED2D0E94AC2419F40E94A02AFF
:10374A000DC0E130A0E0FA0719F40E94A32A06C0CE
:10375A00E230A0E0FA0711F40E94A62A0E94C724C8
:10376A00A1F4E82D0E94AC2419F40E94A02A0DC0ED
:10377A00E130A0E0FA0719F40E94A32A06C0E23059
:10378A00A0E0FA0711F40E94A62A0E94CC2431F57F
:10379A00EC2D0E94AC2419F40E94A02A1FC0E1302B
:1037AA00A0E0FA0719F40E94A32A18C0E230A0E0A8
:1037BA00FA0719F40E94A62A11C0E330A0E0FA071A
:1037CA0029F4EFE6F7E00E94992A08C0E430A0E065
:1037DA00FA0721F4EDE7F7E00E94992A0E94BD2436
:1037EA0021F4E5EBF7E00E94992A0895E0E8EBBBA3
:1037FA00EABBE0E0E8BBEFEFE7BBEFE6E5BBE0E9F9
:10380A00E4BBE0E0E2BBE1BBE0E5E3B9E8E0E2B952
:10381A00E0E0E0936200E0936100E0936500E093EA
:10382A006400E0BFE7E6E3BFE0E0E2BFE1BFE8EA49
:10383A00EFBDECE0EEBDE0E0ECBDE7BDE6BDEAE7DA
:10384A00EBBDE2E1EABDE0E0E9BDE8BDE093790065
:10385A00E0937800E0E1E7BFEBE6E5BDE0E0E4BD38
:10386A00E3BDE1E8E0938B00E5E0E0938A00E0E065
:10387A00E0938900E0938800E0938100E093800060
:10388A00E0938700E0938600E0938500E09384004C
:10389A00E0938300E0938200E0936A00EABFE0E5E8
:1038AA00E9BFE8BFE0E1E7BFE0E0E0937D00EBB904
:1038BA00E8E9EAB9E6E0E0939500E0E0E0939000F9
:1038CA00EFE2E9B9E0E8E8B9E0E0E0BDE3E5EDB947
:1038DA00E0E0EEB9E4E1EA930E94B621EEE1E1BD4F
:1038EA00EEE0E1BD78940E9448210E947429662482
:1038FA0077240E94FC28E1E0E0934905E0E0E093A8
:10390A004A05E1E0E51511F00C94F91D062C07288B
:10391A0011F00C943C1D0E94F728319751F4A89598
:10392A000E94B1280E94A92A0E942F2A0E94B62A20
:10393A00A8950E94F728309711F00C94F81C0E9461
:10394A00B1280E94A92A0E94C12A319729F4A89570
:10395A000E942F2A0E94B62A0E94C12A3B9798F0F9
:10396A00A895AEE1B0E00E947C2C0E94B62A0E9483
:10397A00C62AEA0FFB1F0E94CC2AAEE1B0E00E94E1
:10398A007C2C0E947927E1E0E51569F5A8950E944B
:10399A0003290E94F02938F50E94C12A3197C9F4F7
:1039AA00A8950E9408290E945A28EA0FFB1FE09353
:1039BA002305F09324050E94C12A3A96A4E0B0E0B8
:1039CA000E94942CAC9AECE2F1E00E94D12AA895CC
:1039DA00AC980E94E4270E94F02928F40E94342A15
:1039EA000E94D52AA8950E94C62AEA17FB0718F44E
:1039FA00A8950E94D52A0E947C29CCF50E94D72A34
:103A0A000E94DC2AA8950E94EA2A20F40E94F22A3F
:103A1A00319603C00E94F22A3197FE93EE93A8953D
:103A2A00A0911C05AA2312F40E94F72A0E94FE2ADA
:103A3A0014F00E94062BA0913605AA2312F40E94C4
:103A4A0036240E94C3283197A0913505B0913605D6
:103A5A00EA17FB0734F40E94C328E0933505F09374
:103A6A0036050E940D2B10F00E94152BA8950E9476
:103A7A00C72411F00C94851D0E94B1280E94A92A1E
:103A8A000E942F2A0E94B62A0E947C29CCF50E9405
:103A9A00D72A0E94DC2A0E94C62AEA17FB0710F4DA
:103AAA000E94D52A0E947C295CF50E94D72A0E948E
:103ABA00DC2A0E94EA2A20F40E94F22A319603C0E4
:103ACA000E94F22A3197FE93EE93A0911C05AA2335
:103ADA0012F40E94F72A0E94FE2A14F00E94062B72
:103AEA00A0913605AA2312F40E9436240E94902936
:103AFA0014F00E9498290E940D2B10F00E94152B99
:103B0A000E94CC2411F00C94F91D0E945A28129795
:103B1A0010F40C94F91D0E94B1280E94A92A0E944F
:103B2A002F2A0E94B62A0E947C29CCF50E94D72A05
:103B3A000E94DC2A0E94C62AEA17FB0710F40E9498
:103B4A00D52A0E947C295CF50E94D72A0E94DC2A89
:103B5A000E94EA2A20F40E94F22A319603C00E94A7
:103B6A00F22A3197FE93EE93A0911C05AA2312F430
:103B7A000E94F72A0E94FE2A14F00E94062BA091A6
:103B8A003605AA2312F40E9436240E94902914F0C2
:103B9A000E9498290E940D2B10F00E94152B0E945A
:103BAA00182BD001882799270E942B2EA8F40E944F
:103BBA003D240E9436240E9428240E942F240E9419
:103BCA0074290E94442955240E94452A0E94482AA1
:103BDA000E94482A0E94562A0E942F2AED34A4E005
:103BEA00FA0710F00E947429E1E0E51511F00C942F
:103BFA00FA1E062C072889F4A0913205AA236AF432
:103C0A000E941E2B14F40E94242B0E94DD292CF4FE
:103C1A000E942E2B12F40E943D240E94C22489F491
:103C2A00A0913205AA236AF40E941E2B14F40E9462
:103C3A00242B0E94DD292CF40E942E2B12F40E94C0
:103C4A003D24062C072811F00C947E1E0E94DF28C2
:103C5A000E94F92910F40E943D240E94DF280E9444
:103C6A00F92910F40C947E1E0E94122ABCF40E94B8
:103C7A0017280E94382B0E94DF280E944F2BEA0F38
:103C8A00FB1F0E943F290E94542B20F40E94E42724
:103C9A000E943F290E94592B0E945E2B0E94E22912
:103CAA00309711F40E940B2A0E946C2B20F40E9478
:103CBA00712B319603C00E94712B3197FE93EE93BC
:103CCA00A0911A05AA2312F40E94762B0E947D2B3A
:103CDA0014F00E94852BA0913405AA2312F40E94A5
:103CEA003D240E94232831970E94222A14F40E941C
:103CFA008C2B0E94C224B9F50E94122A7CF40E94DD
:103D0A0017280E94382B0E94542B20F40E94E42783
:103D1A000E943F290E94592B0E945E2B0E94E22991
:103D2A00309711F40E940B2A0E946C2B20F40E94F7
:103D3A00712B319603C00E94712B3197FE93EE933B
:103D4A00A0911A05AA2312F40E94762B0E947D2BB9
:103D5A0014F00E94852B0E94232831970E94222A60
:103D6A0014F40E948C2B0E94CC24A1F50E945F2897
:103D7A000E94222A34F40E945F28E0933305F093CC
:103D8A0034050E94182BD001882799270E942B2ED0
:103D9A00C8F40E943D240E9436240E9428240E94CE
:103DAA002F240E9474290E9444295524A0E2B0E0DD
:103DBA000E947E270E94452A0E94482A0E94482A79
:103DCA000E94562A0E942F2AED34A4E0FA0710F026
:103DDA000E947429E3E0F0E06E167F0630F40E9438
:103DEA00E427309711F40E943D24E1E0E51511F033
:103DFA000C94451F0E94BD2451F5999906C00E9452
:103E0A00922BA5E3B5E00E9496289A9909C00E94D0
:103E1A00922BA5E3B5E0ED91FD913197FE93EE93D8
:103E2A00989904C00E94922B0E94262A9B9904C04A
:103E3A000E94922B0E94262ACF9909C00E94922B97
:103E4A00A3E3B5E0ED91FD913197FE93EE930E94C5
:103E5A00902914F00E9498290E94162AA436E0E0BC
:103E6A00BE0714F00E941B2AA0913605AA2312F459
:103E7A000E943624A0913405AA2312F40E943D24FC
:103E8A000E94B628F301309729F40E947624EDEBBC
:103E9A00F7E023C0E130A0E0FA0729F40E94762473
:103EAA00E7ECF7E01AC0E230A0E0FA0729F40E9432
:103EBA007624E1EDF7E011C0E330A0E0FA0729F437
:103ECA000E947624EBEDF7E008C0E430A0E0FA07A0
:103EDA0041F40E947624ECE5F2E0FA93EA930E9418
:103EEA009421062C072811F00C94D21FE42D0E946D
:103EFA00AC2439F40E94952BE5EEF7E00E948D245C
:103F0A004CC0E130A0E0FA0739F40E94952BE0EFAB
:103F1A00F7E00E948D2441C0E230A0E0FA0739F4AC
:103F2A000E94952BEBEFF7E00E948D2436C0E33018
:103F3A00A0E0FA0739F40E94952BE5E0F8E00E9428
:103F4A008D242BC0E430A0E0FA0739F40E94952BA7
:103F5A00EFE0F8E00E948D2420C0E530A0E0FA07E7
:103F6A0039F40E94952BE9E1F8E00E948D2415C0EE
:103F7A00E630A0E0FA0739F40E94952BE3E2F8E074
:103F8A000E948D240AC0E730A0E0FA0731F40E94AB
:103F9A00952BEDE2F8E00E948D240E94C224F1F4F0
:103FAA00ED2D0E94AC2429F40E94952BE5EEF7E052
:103FBA0011C0E130A0E0FA0729F40E94952BE0EF46
:103FCA00F7E008C0E230A0E0FA0741F40E94952B1E
:103FDA00EBEFF7E0FA93EA930E9494210E94C72438
:103FEA00F1F4E82D0E94AC2429F40E94952BE5EE09
:103FFA00F7E011C0E130A0E0FA0729F40E94952BFE
:10400A00E2EFF7E008C0E230A0E0FA0741F40E94CC
:10401A00952BEBEFF7E0FA93EA930E9494210E9422
:10402A00CC2481F5EC2D0E94AC2429F40E94952B16
:10403A00E5EEF7E023C0E130A0E0FA0729F40E9498
:10404A00952BE2EFF7E01AC0E230A0E0FA0729F474
:10405A000E94952BEBEFF7E011C0E330A0E0FA07DE
:10406A0029F40E94952BE5E0F8E008C0E430A0E0CE
:10407A00FA0741F40E94952BEFE0F8E0FA93EA93ED
:10408A000E9494210E94B6280E946928E7E3F8E07A
:10409A000E948D24A895E0913505F0913605E093AC
:1040AA002B05F0932C050E94292A0E949E27EEE4F4
:1040BA00F8E00E948D2A0E942F2A0E9470280E94EE
:1040CA00942A8CE00E94D22360960E9491240E9436
:1040DA009E270E9487210E94801AE0934505F0934B
:1040EA0046050E94801A9F010E942E270E94581A94
:1040FA008F010E94581AE0934305F09344050E94E9
:10410A00B628A8950E949E27E2E6F8E0FA93EA9379
:10411A00F9010E9470280E946329F8010E94702800
:10412A008CE00E94D22360960E940D290E949E274D
:10413A000E948721A8950E94E229EE0FFF1FE1BF86
:10414A00E0913505F0913605EE0FFF1FE0938600EA
:10415A000E9452293196E3BDA895E4E0F0E06E167C
:10416A007F0690F49A9B07C00E94922B0E94C52753
:10417A003196FE93EE93999B07C00E94922B0E9460
:10418A00C5273197FE93EE930E94C229A233E1E03C
:10419A00BE0770F00E94C229AC32E1E0BE0730F4DB
:1041AA00ECE2F1E0E0932105F09322050E94282435
:1041BA000E942F2A339720F40E9436240E943D241D
:1041CA00552021F49B9902C0CF9BFECF0E94D21AA0
:1041DA00A8950C94861CFFCFFFE0FA95F1F7089595
:1041EA00A1B3AF70A1BB919A9098F6DF929AF4DFCF
:1041FA00A0B39298F1DF929AEFDF9298A7FDF5CFDC
:10420A000895A07FAB2BA2BB929A0E94F1209298AC
:10421A000E94F12008959198A1B3A76FA1BBB2B3F0
:10422A00BF70A881EEDFA881A295EBDF919A0C946A
:10423A00FE23929A0E94F120E0B392980E94F12004
:10424A00E07F08950E94F120F4DFAE2FF2DF91980B
:10425A00E295EA2B08950E94F5200E949B2BEF57C6
:10426A00FA4FE081F0E0DF01E981F0E0EA0FFB1F9D
:10427A00EA930E941021E981E0938505E881E093A1
:10428A008605229608950E94F520E2E0EA930E94AC
:10429A0010210E94F520ECE0EA930E9410210E946E
:1042AA00F520E1E0EA930E941021E0E0E093860520
:1042BA00E09385050895EF93FF93A8816894AA3047
:1042CA0061F0E894E0918505EF5FE0938505E09160
:1042DA008705A0918505EA1760F4E0918605EF5FEE
:1042EA00E0938605E0E0EA93E0918605EA93B3DF7E
:1042FA002EF076DF909AA881AA938DDFFF91EF9135
:10430A000C94FE231A93A981BA81ED91A983BA83E9
:10431A001E2FE03019F01A93CEDFF5CF0EC01A9394
:10432A00E981FA813196E983FA833197E4911E2F64
:10433A00E03019F01A93BFDFF3CF1881239608955E
:10434A00AA27BB271197F1F708959198A1B3A76FF0
:10435A00A1BBB2B3BF70A8810E940621919A0C94A6
:10436A00FE2392989098E881E09387050E949B2B00
:10437A00E058FF4FE09383050E949B2BE054FF4FC8
:10438A00E09384050E949E2B0E949E2B0E949E2BE6
:10439A00D7DFE0E2EA93D9DFD3DFEAE20E94A42B77
:1043AA00E4E00E94A42BE5E80E94A42BA1B3AF701D
:1043BA00A1BB919A0E942721E53019F0E0E00C9404
:1043CA00FE230E94F520E6E0EA930E9410210E9453
:1043DA004821E1E00C94FE235D9BFECFE881ECB915
:1043EA0008C21A930A93AC81BD810E94592C309756
:1043FA00C1F0AA81BB810E94592C8F01309749F0E4
:10440A000230E0E01E0760F0F80131978F01ED936A
:10441A00FC93AC81BD810E9496283197AE81A0831E
:10442A0003C0EE81EA93D8DF19810881279608959F
:10443A0026970E94302E10E0EA89FB893196EA8B92
:10444A00FB8B3197E4912E2FE03011F40C94CE239C
:10445A00E12F0E94AC2439F4253211F411E002C094
:10446A000E94A92B95C1E130A0E0FA07A9F42532F0
:10447A0019F40E94A92B8BC112E040E000E02D3212
:10448A0011F401E085C12B3211F44BE281C12032D3
:10449A0011F440E27DC104C0E230A0E0FA0761F401
:1044AA0050E013E0203339F40E94B42BE0E8F0E046
:1044BA00EA2B0E2F6DC106C0E330A0E0FA0711F017
:1044CA000C94CD23203310F02A3308F015C0A52F01
:1044DA00B0E0EAE0F0E0EA02F0015E2F652F77270C
:1044EA00A22FB0E0E0E3F0E00E94712CEA1BFB0B84
:1044FA00DB01EA0F5E2F4CC10E94B72BE336A0E026
:10450A00FA0749F40E94BA2BE889F989A481AA9387
:10451A000E94C02B3CC1E337A0E0FA0741F40E9495
:10452A00BA2B0E94CA2B0E9400241E2F11C0E0370A
:10453A00A0E0FA07D9F40E94BA2B0E94CA2B0E9463
:10454A000A241E2F0E94B42BE8E0F0E0EA2B0E2F7B
:10455A000E94B42BE2E0F0E0EA2B0E2F0E94B42B6B
:10456A00EFE7FFEFEA230E2F30E04FC0E436A0E07A
:10457A00FA0721F0E936A0E0FA0739F40E94B42BD1
:10458A00E4E0F0E0EA2B0E2F04C0E537A0E0FA07DA
:10459A0031F4ECE8F0E0EE83FF8315E016C0E8356D
:1045AA00A0E0FA0739F40E94B42BE8E0F0E0EA2B25
:1045BA000E2F06C0E837A0E0FA0711F00C94CC23BE
:1045CA00E6E9F0E0EE83FF8314E00E94B42B0E9438
:1045DA00D42BB9F00E94BA2B0E94DA2BAB85AA23FE
:1045EA003AF4EA85FB850E941C2CEA87FB874DE298
:1045FA00403011F01F5F04C00E94B42B0E94E22BCE
:10460A0004C00E94BA2B0E94DA2B0E94E72BE9F41D
:10461A001517D8F40E94B42BE0E8F0E0EA23FB2354
:10462A00309771F00E94B42B0E94D42B39F00E946B
:10463A00B42B0E94E22B242F115001C020E301C0A9
:10464A0020E20E94A92B5150E3CF312F0E94B42BB4
:10465A00E2E0F0E0EA23FB23309701F13030E9F0A1
:10466A000E94B42BE8E0F0E0EA23FB23309741F004
:10467A00EE81FF813196EE83FF833197E49105C085
:10468A00AE81BF81ED91AE83BF83EA930E94C02BB6
:10469A00503009F051503150E1CF6EC020E3EE8125
:1046AA00FF810E945D2CE887F987EE81FF813296AF
:1046BA00EE83FF83E885F985AA85BB85AE17BF0718
:1046CA0050F02F5FA885B985EA85FB85EA1BFB0BAD
:1046DA00EA87FB87EFCF2A3380F00E94B42BE8E009
:1046EA00F0E0EA23FB23309721F00E94B72B37969C
:1046FA0003C00E94B72BB7962E2F0E94B42BE0E17D
:10470A00F0E0EA23FB23309761F5213320F4A885F2
:10471A00B985119709F410C0531718F00E94E72BB6
:10472A0009F024C020E20E94B42BE0E8F0E0EA237A
:10473A00FB233097B1F020E3A02FB0E0E0E1F0E0F6
:10474A00EA2B0E2F0E94B42B0E94D42B51F00E9408
:10475A00B42B0E94E22B4A930E94C02B503009F0DE
:10476A0051500E94A92B503009F051503150A88560
:10477A00B985129708F092CF0E94E72B41F050308A
:10478A0031F05150E0E2EA930E94C02BF8CF10E0DA
:10479A0053CE0E94372E64960895FF920E94EB2B07
:1047AA00DE0116960E94F42BEA83FB83DE0114963F
:1047BA000E94F42B0E94F92BAA81BB81E0E0EC93C2
:1047CA000CC0FF920E94EB2BE0E0EA83EB83DE0150
:1047DA0014960E94F42B0E94F92B198108812496C1
:1047EA00FF900895E881EFB9EEB1F0E0E078E1F3E7
:1047FA00EFB121960895A991B991EE27FF276D91FE
:10480A00662311F03196FBCF0895AA27BB27E991B9
:10481A00F9910590002011F01196FBCFFD01089542
:10482A000A921A92FA926A937A938A939A93AA9319
:10483A00BA93EA93FA93EFB7EA930895A9E2B1E03B
:10484A000E94802C0895E0E0F0E0E0932105F093C7
:10485A0022050895E0E0F0E0E0932305F0932405B3
:10486A000895E0E0F0E0E0933505F0933605089509
:10487A00E0E0F0E0E0933305F09334050895AA24CC
:10488A00BB245524ACE1B0E0E0E0F0E00E94942CB7
:10489A00AEE1B0E00E94942CAC9AE4EFF1E0FA9316
:1048AA00EA930E94072CAC98E4EFF1E0FA93EA93BA
:1048BA000E94072CAC9AE4EFF1E0FA93EA930E9483
:1048CA00072CAC98E4EFF1E0FA93EA930E94072CE4
:1048DA00AC9AE4EFF1E0FA93EA930E94072CAC98C1
:1048EA000895E0E0EA93EA930C943021EEE4F1E0D3
:1048FA00FA93EA930E949421E0E0EA930895E3E0B0
:10490A00EA930E943021F2CFE1E0EA930C9430213D
:10491A00FA93EA930C949421E0E0EA93E2E0EA93B2
:10492A000C943021A0E0B0E00E94802C0895E15060
:10493A000E949C2CEF5F0895EEE1F0E0FA93EA936F
:10494A000C94072CEF5F0E949C2CE1500895F0E034
:10495A00309708950E944821E4EFF1E0FA93EA9330
:10496A000C94072CE0E0EA93CACFEEE4F1E0D0CF52
:10497A00E4E0F0E0E615F7050895E1E0F0E0E61579
:10498A00F7050895E2E0F0E0E615F7050895E3E09B
:10499A00F0E0E615F7050895E6E8F2E0B9CFA4E3FA
:1049AA00B0E00E947C2CE0932305F0932405A2E357
:1049BA00B0E00E947C2CE0932105F0932205A0E54B
:1049CA00B0E00E947C2CAEE2B0E00E94942CA6E5F6
:1049DA00B0E00E947C2CA0E1B0E00E94942CACE5EF
:1049EA00B0E00E947C2CAEE0B0E00E94942C0895C6
:1049FA000E947C2CA2E1B0E00E94942C0895A6E3C8
:104A0A00B0E00E947C2CA8E0B0E00E94942C0895AB
:104A1A000E947C2CAAE0B0E00E94942C08950E9487
:104A2A007C2CACE0B0E00E94942C0895A5E1B1E0A2
:104A3A000E947C2CE0933905F0933A05A5E0B1E099
:104A4A0008950E947C2CE0933705F0933805089569
:104A5A00EBE9F2E05DCFAEE3B0E00E947C2CE0939C
:104A6A002305F0932405ACE3B0E00E947C2CE0938C
:104A7A002105F0932205A2E5B0E00E947C2CAEE26B
:104A8A00B0E00E94942CA8E5B0E00E947C2CA0E142
:104A9A00B0E00E94942CAEE5B0E00E947C2CAEE01F
:104AAA00B0E00E94942C0895A0E4B0E00E947C2C0F
:104ABA00A8E0B0E00E94942C0895A7E1B1E00E941A
:104ACA007C2CE0933905F0933A05A7E0B1E008950C
:104ADA00E0EBF2E01DCFA8E4B0E00E947C2CE0936A
:104AEA002305F0932405A6E4B0E00E947C2CE09311
:104AFA002105F0932205A4E5B0E00E947C2CAEE2E9
:104B0A00B0E00E94942CAAE5B0E00E947C2CA0E1BF
:104B1A00B0E00E94942CA0E6B0E00E947C2CAEE0AB
:104B2A00B0E00E94942C0895AAE4B0E00E947C2C84
:104B3A00A8E0B0E00E94942C0895A9E1B1E00E9497
:104B4A007C2CE0933905F0933A05A9E0B1E0089589
:104B5A00AAE6B0E00E947C2CE0932305F09324059A
:104B6A00A8E6B0E00E947C2CE0932105F093220590
:104B7A00ACE6B0E00E947C2CAEE2B0E00E94942C3D
:104B8A00AEE6B0E00E947C2CA0E1B0E00E94942C3A
:104B9A00A0E7B0E00E947C2CAEE0B0E00E94942C2A
:104BAA000895A4E7B0E00E947C2CA8E0B0E00E943F
:104BBA00942C0895ABE1B1E00E947C2CE093390576
:104BCA00F0933A05ABE0B1E00895ACE7B0E00E949B
:104BDA007C2CE0932305F0932405AAE7B0E00E9419
:104BEA007C2CE0932105F0932205AEE7B0E00E9409
:104BFA007C2CAEE2B0E00E94942CA0E8B0E00E94C7
:104C0A007C2CA0E1B0E00E94942CA2E8B0E00E94C3
:104C1A007C2CAEE0B0E00E94942C0895A6E8B0E0A7
:104C2A000E947C2CA8E0B0E00E94942C0895ADE18B
:104C3A00B1E00E947C2CE0933905F0933A05ADE08F
:104C4A00B1E00895AEE8B0E00E947C2CE093230521
:104C5A00F0932405ACE8B0E00E947C2CE093210597
:104C6A00F0932205A0E9B0E00E947C2CAEE2B0E00D
:104C7A000E94942CA2E9B0E00E947C2CA0E1B0E052
:104C8A000E94942CA4E9B0E00E947C2CAEE0B0E033
:104C9A000E94942C0895A8E9B0E00E947C2CA8E018
:104CAA00B0E00E94942C0895AFE1B1E00E947C2C00
:104CBA00E0933905F0933A05AFE0B1E00895A0EA30
:104CCA00B0E00E947C2CE0932305F0932405AEE922
:104CDA00B0E00E947C2CE0932105F0932205A2EA21
:104CEA00B0E00E947C2CAEE2B0E00E94942CA4EAD0
:104CFA00B0E00E947C2CA0E1B0E00E94942CA6EACD
:104D0A00B0E00E947C2CAEE0B0E00E94942C0895A2
:104D1A00AAEAB0E00E947C2CA8E0B0E00E94942CA1
:104D2A000895A1E2B1E00E947C2CE0933905F0934A
:104D3A003A05A1E1B1E00895A2EBB0E00E947C2C13
:104D4A00E0932305F0932405A0EBB0E00E947C2CAD
:104D5A00E0932105F0932205A4EBB0E00E947C2C9D
:104D6A00AEE2B0E00E94942CA6EBB0E00E947C2C4C
:104D7A00A0E1B0E00E94942CA8EBB0E00E947C2C49
:104D8A00AEE0B0E00E94942C0895ACEBB0E00E9433
:104D9A007C2CA8E0B0E00E94942C0895A3E2B1E034
:104DAA000E947C2CE0933905F0933A05A3E1B1E027
:104DBA000895E4EFF1E0FA93EA930E94072C0C9429
:104DCA004821A2ECB0E00E947C2CE0932305F093EA
:104DDA002405A5ECB0E00E947C2CAEE2B0E00E9473
:104DEA00942CA7ECB0E008950E947C2CAEE0B0E0D1
:104DFA000E94942C08950E94802CA2E1B0E0F0E079
:104E0A000E94942C0895A9ECB0E00E947C2CE093B7
:104E1A002305F0932405ACECB0E00E947C2CAEE2B2
:104E2A00B0E00E94942CAEECB0E00895A0EDB0E0A2
:104E3A000E947C2CE0932305F0932405A3EDB0E0B7
:104E4A000E947C2CAEE2B0E00E94942CA5EDB0E06A
:104E5A000895E8ECF0E0FA93EA930C94072CA7ED96
:104E6A00B0E00E947C2CE0932105F0932205A9ED85
:104E7A00B0E008950E947C2CA0E1B0E00E94942C3E
:104E8A0008950E947C2CE0932105F0932205089551
:104E9A00A5EEB0E00E947C2CE0932305F093240554
:104EAA00A7EEB0E0A1CF0E947C2CA3EEB0E00E9456
:104EBA00942C08950E947C2CE0932305F0932405FA
:104ECA000895EDE6F3E024CDEBE4F5E0FA93EA93F6
:104EDA000C948721A6E0B0E00E947C2C08953197BB
:104EEA000E94942C3196089531960E94942C319701
:104EFA000895E0E0F0E00E94942C0895659785E11A
:104F0A00A0E0B0E00895FE01FA93EA930E94872197
:104F1A0065960895A1E0B0E00E94802C0895A2E071
:104F2A00B0E00E94802C0895A3E0B0E00E94802C9B
:104F3A000895E0E0F5E0FA93EA930895E2E8F3E0F1
:104F4A00FA93EA93E0912105F091220566277727E3
:104F5A000E94612C84E00E94D2232896E2E0EA9320
:104F6A00E3E0EA930E943021E4CF0E948721E0E047
:104F7A00EA93CACCE1E9F3E0CBCCE6EAF3E0C8CCA9
:104F8A00A1E2B5E0ED91FD9108953197FE93EE937C
:104F9A00E2E3F0E0FA93EA930C94072C3196FE933D
:104FAA00EE93E2E3F0E0FA93EA930C94072CA091D3
:104FBA002105B0912205AD32E1E0BE070895E091E6
:104FCA002105F09122050895E2E8F3E0FA93EA93C5
:104FDA000895A3E0B1E00E947C2C08956627772704
:104FEA000E94612C84E00E94D2232896E2E0EA9390
:104FFA00E3E0EA930E9430219CCFE2E3F0E0FA93E7
:10500A00EA930C94072CEBEBF3E0FA93EA93A0E112
:10501A00B0E00E947C2CE2CFEFECF3E079CCE4EE36
:10502A00F3E076CCA0E1B0E00E947C2C0895A0E1E8
:10503A00B0E0EFE0F0E00E94942C0895E09137058B
:10504A00F091380508950E94342C0E94612C84E066
:10505A000E94D2232896E2E0EA93E3E0EA930E94D0
:10506A00302167CFED91FD9190CFED91FD9196CFD3
:10507A00E4E6F0E0E0933705F09338050895E0910F
:10508A002305F09124050895E9E1F4E041CCA3E277
:10509A00B5E0E8CFA3E2B5E0E8CFA0912305B0914F
:1050AA002405AB3EE1E0BE070895A0912305B09127
:1050BA0024050895A3EEB0E00E947C2C0895E4E64E
:1050CA00F0E00E94942C0895E0E0EA931DCCE3E01E
:1050DA00EA930C943021662777270E94612C089561
:1050EA0088E00E94D2232C960895A6E1B0E00E949F
:1050FA00782C0895ED91FD913197FE93EE93F5CFBB
:10510A00E130A0E0FA07A0E06A07A0E07A07089574
:10511A00A6E1B0E0E0E0F0E060E070E00E948C2CF4
:10512A000895ED91FD913196FE93EE930895A6E1CF
:10513A00B0E00E948C2CADE1B5E00895E0931D0526
:10514A00F0931E050895EBEBF3E0FA93EA93AEE0D1
:10515A00B0E00E947C2C42CFAEE0B0E00E947C2CF2
:10516A000895E4E6F0E0FA93EA930C94072CAEE093
:10517A00B0E0EFE0F0E00E94942C0895E091390548
:10518A00F0913A050895E4E6F0E0E0933905F093EA
:10519A003A050895E6EBF4E0FA93EA93AEE2B0E05A
:1051AA000E947C2C98CF84E00E94D2232896E0E0CB
:1051BA00EA938DCFAEE2B0E00E947C2C0895A2E182
:1051CA00B0E00E947C2C0895A2E1B0E092CEE5E026
:1051DA00F5E09ECBEAE1F5E09BCBA2E1B0E00E94CC
:1051EA00802C0895A8E0B0E00E947C2C0895A4E0E9
:1051FA00B0E0E1E0F0E00E94942C0895AAE0B0E06B
:10520A000E947C2C0895ACE0B0E00E947C2C0895AA
:10521A00E0E0EA935CCFAAE2B0E00E947C2C089519
:10522A0084E00E94D223289677CBACE2B0E00E94B9
:10523A007C2C0895A4E1B0E00E947C2C0895E2EC55
:10524A00F1E00E94942C0895E1E0F0E00E94942C91
:10525A000895E6E1F0E00E94942C0895EFE0F0E072
:10526A000E94942C0895E0E0F0E0E0931105F09399
:10527A0012050895E0931705F09318050895ACE117
:10528A00B0E037CEE0E0F0E0E0931905F0931A05BC
:10529A00E0931B05F0931C050895A7E2B1E00E9474
:1052AA007C2C0895E2E6F6E033CBE7E7F6E030CB74
:1052BA00EBE8F6E0FA93EA93E2DE0DCF80DE0BCF5D
:1052CA000E948721E1E05E2EAA24BB24D8CFE5E91B
:1052DA00F6E0FA93EA93F2CFA0E3B0E00ACEAAE1AD
:1052EA00B0E007CEA0914505B09146050895A0917A
:1052FA002D05B0912E050E94272E0895E0913505BF
:10530A00F09136053F97E0933505F0933605A09165
:10531A003605AA230895A0913505B0913605A4361D
:10532A00E0E0BE070895E4E6F0E0E0933505F09387
:10533A0036050895E0914505F091460508959FDEEA
:10534A00D1DFAE17BF070895A0E2B0E00E947C2C1F
:10535A00CBCDE0914305F09144050895A091430512
:10536A00B09144050895A0913105B0913205089590
:10537A00E0914705F09148050895A0912105B09163
:10538A0022050895AE0FBF1FEAE0F0E00E943E2C0E
:10539A00DF01E3E2F0E00E94462CE0933305F0934C
:1053AA003405E6DF3A96E0934705F09348050895F9
:1053BA00DADFAD3FEFEFBE070895E0913305F091D4
:1053CA00340508957497E0933305F0933405A0915A
:1053DA003405AA230895C2DFEA17FB070895ACE152
:1053EA00B0E00E947C2C80CDB9DFAE17BF070895CC
:1053FA00A0E3B0E00E947C2C0895AC9AE0E9F1E0C9
:10540A00FA93EA930E94072CAC980895E3E2F0E03D
:10541A00E0933305F09334050895A5DF0E94272E03
:10542A000895A0913305B09134050895E4E6F0E0BB
:10543A00E0933305F09334050895F3DFEA17FB0789
:10544A000895A3E3B5E06DCEB8DFE0932905F093A4
:10545A002A050895AAE1B0E00E947C2C08956ADF2B
:10546A00E0932305F09324050895E0E9F1E0FA9327
:10547A00EA930C94072CA4E6B0E00E943E2C08950F
:10548A00AA24BB2429CFAC9AE4EFF1E0FA93EA9379
:10549A000E94072CAC98E4EFF1E0FA93EA930C949B
:1054AA00072CAC9AE4EFF1E0FA93EA930E94072CF6
:1054BA00AC980895E3E5EDB9E0E0EEB9B99ABA9A85
:1054CA00BB980895E0E0EA930E94F723F0E008957C
:1054DA0066277727DF01CB01E8E00E94282C089590
:1054EA00662777270E94172C8F01087F1F7716954A
:1054FA000795169507951695079508950E94342CD9
:10550A000E94132D089584E00E94E62326960895AA
:10551A00FA93EA93E0912B05F0912C05DCCDE0910A
:10552A002905F0912A05D7CDFA93EA9380E00E94E3
:10553A00E62322960895EAE4F7E0F6CFE8E5F7E0F5
:10554A00F3CFE1E6F7E0F0CFDF01EAE0F0E00E9416
:10555A00462CD4DFA3E1B5E00E94DA2CED93FC934C
:10556A000895A0911305B09114050E943E2CE09372
:10557A001105F09312050895A4E0B0E00E947C2C76
:10558A0008957DDDA0911105B09112050895E0936B
:10559A001105F09312050895FA93EA930C94072CD7
:1055AA006EDDF5CFE0911105F091120564CFDF01B0
:1055BA00E0911B05F0911C05E650FF4F0E94462C16
:1055CA00E0933505F09336050895B4DEA0911105F0
:1055DA00B0911205AE17BF070895ABE1B5E0ED91A2
:1055EA00FD910895E0E0F0E0E0931B05F0931C05BF
:1055FA000895A0911B05B0911C05AD32E1E0BE07EC
:10560A000895ECE2F1E0E0931B05F0931C05089580
:10561A00A0911105B0911205A33CE1E0BE070895DF
:10562A00E2ECF1E0B4CFA0E2B0E00E947C2C0F01E2
:10563A005CCD99DEEDEFFFEFEA17FB0708959DDEDB
:10564A00E5E0F0E00E94462CE0933305F093340540
:10565A000895B3DE7E97E0933305F0933405A09165
:10566A003405AA230895DF01EAE0F0E00E94462CFF
:10567A0045DFA5E1B5E00E94DA2CED93FC93ACE19D
:10568A00B0E00E947C2CA0911505B09116050E94ED
:10569A003E2CF0CDA0911705B091180508958FDC26
:1056AA00F9DFEA17FB070895E0911705F09118054D
:1056BA00E2CEDF01E0911905F0911A05EA56FF4F93
:1056CA000E94462CE0933305F0933405089541DE99
:1056DA00E1DFAE17BF070895A9E1B5E0ED91FD91AD
:1056EA000895E0E0F0E0E0931905F0931A050895B3
:1056FA00A0911905B0911A05AD32E1E0BE070895EF
:10570A00ECE2F1E0E0931905F0931A05089596DCAE
:10571A00E0933305F09334050895E9E1F0E03CCFD6
:10572A00EAE0EA93E0E0EA930C943021E881F0E0C1
:10573A0008950E94A521E0E3EA930C94AA21EA9332
:10574A000E9410210C94A5212A93EF85F889FA93D7
:10575A00EA93FE013F96FA93EA930C94F621A02F5E
:10576A00B0E00895E22FF0E00895E889F9893497C6
:10577A00E88BF98B0895EF85F889FA93EA93FE018D
:10578A003F96FA93EA930C94F621A889B98914965C
:10579A000E94592CEE83FF83FA93EA930895E4E07A
:1057AA00F0E0EA23FB2330970895A889B989149673
:1057BA000E94592CEA87FB870895EBEFFFEFEA2353
:1057CA000E2F0895E02FF0E0E1700895F82E229749
:1057DA001A930A93DE010E94132C8D0108950E94E8
:1057EA00132C0E94592C0895FA93EA931A930A9358
:1057FA00FE013696FA93EA93E0E0F0E0FA93EA9330
:10580A000C941D22E991F991309639F083E397E0DF
:10581A000197F1F7A8953197C9F708950024AF0DBC
:10582A00B01D0895EA2BFB2B682B792B0895F1956F
:10583A00E195F0400895F09560957095E195FF4FD8
:10584A006F4F7F4F0895EE230E2EFD01BC0131F0FC
:10585A00EE0FFF1F661F771F0A94D1F708956F2F67
:10586A00660F660B762F08958B2F880F880B982F5B
:10587A000895FA9FF02DEB9FF00DEA9FE02DF10DB0
:10588A0008950024112490E1AA0FBB1F001C111CCB
:10589A000E1A1F0A18F40E0E1F1E01C0A1609A9557
:1058AA0099F7FD01D0010895ED91FC9111970895A2
:1058BA000590F491E02D08957A936A93FA93EA9306
:1058CA000895689401C0E89401D0A9D0182E862FB3
:1058DA00612D192E972F712D1B2EBF2FF12D1A2EE8
:1058EA00AE2FE12D0895129602D0BF01129711969C
:1058FA0002D0FE2F1197E199FECFFF93FFB7F894DC
:10590A00AEBBBFBBE09AEDB3FFBFFF91089507D0CE
:10591A0012960F01FB0103D0F0011297089507D0E8
:10592A001196EF93EF2F03D0EF9111970895E19B12
:10593A0002C0A895FCCF9FB7F894AEBBBFBBE09A54
:10594A008DB3E81719F0EDBBE29AE19A9FBF08956B
:10595A00552342F4503811F4E0FF04C03196691F10
:10596A00791F6BF050E8572711F45F93C6C05F3F69
:10597A0031F0660F000C57956795752F08955F9360
:10598A0000200AF0C6C0BFC050E8192E1522880FA1
:10599A00991F9527550F879550E8072E0522660F00
:1059AA00771F7527550F67950895689401C0E89485
:1059BA005F93F2DF703818F07F3F08F49EC056E11B
:1059CA00571BAAF4519558300EF4593030F0EFEFC6
:1059DA00FFEF6FEF7FE777F91AC077275523B9F002
:1059EA00EE0FFF1F661F771F5A95D1F710C0772752
:1059FA00583028F0EF2FF62F672F5850F9CF55233C
:105A0A0031F076956795F795E7955A95D1F7002085
:105A1A000AF411DF5F910895689401C0E894309701
:105A2A0060407040B1F0002426F0772312F400940D
:105A3A0002DF172E7EE1112032F07A95EE0FFF1F5A
:105A4A00661F111CF9CFEF2FF62F612D5F938ADFA6
:105A5A005F9108954F93AF01FD01DA01AB01BC01DB
:105A6A00CA01402D012C142E4F910895EA0FFB1FF5
:105A7A00681F0895E095F0956095EF5FFF4F6F4FAF
:105A8A0008955F9381DF903839F1703821F1572FEB
:105A9A00591B13F112F4DEDFFACF583118F0AA2796
:105AAA00BB278827583028F0AB2FB82F88275850A3
:105ABA00F9CF552329F08695B795A7955A95D9F721
:105ACA00502D512562F0D2DF38F46795F795E795A6
:105ADA00739513F41EC0BEDF45DF5F910895EA1B7C
:105AEA00FB0B680B51F010F40094C4DF6623A2F399
:105AFA00EE0FFF1F661F7A95CBF7EE27FF27662763
:105B0A0077275F910895EFEFFFEF6FE77FEF5F91E0
:105B1A000895EFEFFFEF6FE77FE75F9108955F93D7
:105B2A0033DF703851F3903841F301240894791F18
:105B3A0023F41CF300203AF3ECCF0F921F932F9318
:105B4A003F934F93112722279927689FA0018F9F80
:105B5A00302D410D591F6B9F300D411D591F8E9FCE
:105B6A0027D0BF9F25D06A9F23D0BE9F1DD0AF9F4D
:105B7A001BD0AE9F110D291F391F491F591FE32F33
:105B8A00F42F652F522F4F913F912F911F910F9014
:105B9A0066232AF0550FEE1FFF1F661F02C073957A
:105BAA004BF2D6DE5F910895100D211D391F02C0F8
:105BBA00200D311D491F591F08955F93E5DE703886
:105BCA0021F411200AF49FCFA4CF903809F495CF7D
:105BDA0001240894970B1BF4D4F30020F3CF792FF8
:105BEA001F932F933F934F93112411272227332773
:105BFA004427552790E2AE17BF078607410730F0C2
:105C0A00AE1BBF0B860B410B089401C08894551F2D
:105C1A00221F331F111CAA1FBB1F881F441F9A95DE
:105C2A0051F7F901612D4F913F912F911F916623F1
:105C3A0032F0550FEE1FFF1F661F7A9543F288DE7A
:105C4A005F91089500240A160B060895EA17FB07C8
:105C5A006807790708955A934A933A932A931A93AD
:105C6A000A9308955D814C813B812A8119810881BB
:105C7A000895AC0FBD1F05900D928A95E1F708951E
:00000001FF
